:020000040800F2
:1000000038110020010100085B380008B9280008F9
:1000100059380008350F0008396400080000000056
:100020000000000000000000000000002949000856
:10003000871A000800000000C53D0008294C000890
:100040001B010008B93B00081B0100081B01000848
:100050001B0100081B0100081B0100081B01000810
:100060001B0100081B0100081B0100081B01000800
:100070001B0100081B010008091500081B010008EE
:100080001B0100081B0100083D0700081B010008B8
:100090001B0100081B0100081B0100081B010008D0
:1000A000994C0008854D00081B0100081B01000841
:1000B000894D000875500008D15200081B01000846
:1000C0001B0100081B0100081B0100081B010008A0
:1000D0001B010008315F00081B0100081B0100081C
:1000E0001B0100081B0100081B010008DFF80CD0F1
:1000F00000F0E6FA00480047897500083811002032
:100100000648804706480047FEE7FEE7FEE7FEE7B1
:10011000FEE7FEE7FEE7FEE7FEE7FEE7494C0008E4
:10012000ED0000082DE9F0410024061B254671F181
:10013000000605DA01240027D0EB070067EB010178
:10014000161E73F1000605DA0027D2EB070201251F
:1001500067EB030300F0D0F986460E4617469C462F
:10016000AC4204D00025D0EB050E65EB010624B1AE
:100170000020D2EB000760EB030C704631463A4694
:100180006346BDE8F08140EA01039B0703D009E024
:1001900008C9121F08C0042AFAD203E011F8013B73
:1001A00000F8013B521EF9D2704780EA010210B5F7
:1001B00002F00043400022D04A001FD0010E01EBA4
:1001C0001261C0F35600C2F3560240F4000042F43C
:1001D0000002A0FB022000047F39140400D0401C60
:1001E00050EA124001D44000491EC2B20C0604EB92
:1001F000D010401C4008802A02D003E0002010BD2F
:1002000020F00100002900DA0020184310BD2DE97C
:10021000FE4F81EA030404F0004421F00041009401
:100220004FF0000B23F0004350EA01045ED052EA85
:1002300003045BD0C3F30A54C1F30A552C44A4F25F
:10024000F3340194A0FB0254C1F3130141F4801173
:10025000C3F3130343F4801301FB024400FB034E7A
:10026000840A970A44EA815447EA8357A4FB076843
:1002700002958D0A05FB07854FEA932C04FB0C546D
:100280002705029D4FEA065847EA1637B5EB0805E1
:100290006EEB070C870E920E47EA811742EA831233
:1002A000A7FB0201B6EB0B0164EB00042B0D43EA44
:1002B0000C335E1844EB1C50DA465146E7FB020152
:1002C000C5F313044FEA0B3343EA14534FEA0432E5
:1002D000019C43EA0603A4F10C040294009CCDE9BE
:1002E00000B400F09FF903B0BDE8F08F0020014694
:1002F000F9E72DE9F04D81EA030404F0004B21F009
:10030000004514464FF0000A23F0004150EA050270
:1003100020D054EA01021DD0C5F30A570246C5F3A6
:100320001303C1F31300C1F30A5640F4801543F4DC
:100330008013A7EB0608101BD64608F2FD3873EBB6
:10034000050002D308F1010801E092185B41B8F101
:10035000000F03DA00200146BDE8F08D00204FF4C5
:100360008011064684460EE0171B73EB050705D384
:10037000121B63EB050306434CEA010C49084FEAE4
:10038000300092185B4150EA0107EDD152EA0300B8
:1003900012D082EA040083EA0501084305D0101B4D
:1003A000AB4106D20122002306E000224FF00043B9
:1003B00002E06FF0010253101AEB06004CEB0851FB
:1003C00010EB0A0041EB0B01BDE8F04D00F01BB94A
:1003D00070B521F0004303430CD0C1F30A5500244B
:1003E000D5EB040564EB0403D617AD1AB34102DB69
:1003F0000020014670BD201841EB025170BDC10FB5
:1004000080EAE0700844CA079623002100F0CDB8C6
:1004100096230022114600F0C8B80EB5C10F80EA3D
:10042000E0700844CA07002140F233438DE80E0013
:100430000A460B4600F0F6F803B000BD0EB540F2D8
:10044000334102910021CDE900110A460B4600F02C
:10045000E9F803B000BD00F0004220F00040C10DFB
:10046000C0F3160040F400007F2901DA0020704735
:10047000962903DCC1F19601C84001E09639884015
:10048000002AF4D04042704770B5C1F30A5201F01F
:1004900000450024C1F3130140F2FF3341F4801101
:1004A0009A4201DA002070BD40F233439A42A2F230
:1004B000334203DC524200F05FF800E090402C43EE
:1004C000F1D0404270BDC1F30A5210B5C1F313011F
:1004D00040F2FF3341F480119A4201DA002010BD4E
:1004E00040F233439A42A2F2334203DC524200F01C
:1004F00043F810BD904010BD2DE9F05F0546002087
:1005000092469B4688460646814640241BE0284684
:1005100041464746224600F02FF853465A46C01A35
:10052000914110D311461846224600F016F82D1AB4
:1005300067EB01084F4622460120002100F00DF82C
:1005400017EB00094E41201EA4F10104DFDC4846F0
:1005500031462A464346BDE8F09F202A04DB203A74
:1005600000FA02F1002070479140C2F1200320FA06
:1005700003F3194390407047202A04DB203A21FA04
:1005800002F00021704721FA02F3D040C2F12002AC
:1005900091400843194670470029A8BF7047401C86
:1005A000490008BF20F00100704710B4B0FA80FC89
:1005B00000FA0CF050EA010404BF10BC704749B1C6
:1005C000CCF1200421FA04F411FA0CF118BF012136
:1005D00021430843A3EB0C01CB1D4FEA00614FEA16
:1005E000102042BF002010BC704700EBC3501044E5
:1005F0000029A4BF10BC7047401C490008BF20F070
:10060000010010BC704710B5141E73F1000408DA25
:10061000401C41F1000192185B411A4301D120F0C6
:10062000010010BD2DE9F04D92469B4611B1B1FA83
:1006300081F202E0B0FA80F220329046FFF78DFF9F
:1006400004460F4640EA0A0041EA0B0153465A4667
:10065000084313D0114653EA010019D0C8F14002F3
:100660005046FFF789FF05460E465046594642461A
:10067000FFF773FF084305D0012004E02046394608
:10068000BDE8F08D0020054346EAE0762C43374371
:100690000A986305E40AA0EB08000022FD0A44EA78
:1006A00047540A3002D500200146E9E70105101938
:1006B0006941DDE9084500196941BDE8F04DA2E74F
:1006C000064C074D06E0E06840F0010394E807009F
:1006D00098471034AC42F6D3FFF70CFD7098000831
:1006E0009098000870B58C1810F8015B15F007039E
:1006F00001D110F8013B2A1106D110F8012B03E0BB
:1007000010F8016B01F8016B5B1EF9D12B0705D4C2
:100710000023521E0DD401F8013BFAE710F8013B0B
:10072000CB1A921C03E013F8015B01F8015B521E27
:10073000F9D5A142D8D3002070BD000070B54C4C53
:100740004FF490652946204600F015FA002864D041
:100750002946204600F0A2F846490888401C088037
:100760000121204600F0E6FA434942F21072B1F846
:100770005800904202D2401CA1F8580007F0E8F857
:100780003E4DB5F91410B5F9120005F0A9FF3C4C27
:10079000A5F856002080A16820468847A088A5F8C3
:1007A000580003F0C3F807F0CFF9364E364C3078D6
:1007B000082833D045F6AC30606042F6EF60A060A8
:1007C00042F2C400E0603148008A2080208E6080C0
:1007D000A16B2D488847208E69882D4C08444FF620
:1007E000FF7101EA80006887207A4FF0000540071A
:1007F0001DD501F0D7FA274949F6A24008802648BE
:1008000040F21A62C188491C89B2C180914204D366
:10081000A16821F00401A160C58070BD41F2130000
:1008200060604FF48060A06040F61B50CAE73078EB
:100830000A2818D2DFE800F0170613050A050D177D
:100840001113EAE7BDE8704006F0F4B808F04AF981
:1008500005E0BDE8704002F0B3BD06F071FCBDE8F4
:10086000704007F0C9BA00F0FDFB84F8B65070BDC7
:1008700000240140340700204801002064000020CB
:10088000540700202B070020E40000200002002075
:10089000B0020020442C0140700900206FEA1121B1
:1008A000016070470029816802D041F0010101E038
:1008B00021F00101816070470029816802D041F474
:1008C000807101E021F48071816070472DE9F04171
:1008D000824E92B0304600F00BF90BA800F039FAC6
:1008E00001214FF4C06003F001FB00248DF831407A
:1008F0004FF46020CDE90D044FF4A0204FF009081B
:100900000B9001278DF83C808DF830700BA9304694
:1009100000F080F9724D8DF831408DF830708DF80F
:100920003C700BA9284600F075F901231A460F21E7
:10093000304600F0C0F9022201231146304600F093
:10094000BAF9012303220021304600F0B4F9012353
:1009500004221946304600F0AEF9012305220B218E
:10096000304600F0A8F9012306220421304600F0A9
:10097000A2F9012307220821304600F09CF9012347
:1009800008220321304600F096F9012309220A21AA
:10099000304600F090F90121304600F084F9012141
:1009A000284600F080F901231A460521304600F060
:1009B00055F901231A460621284600F04FF9002177
:1009C000304600F0CBF84FF4E041284600F0C6F87E
:1009D0000121304600F0B8F80121284600F0B4F8B3
:1009E0000121304600F0A6F80121284600F0A2F8C7
:1009F0000121304600F09EF90121284600F09AF9C5
:100A000040F61451374804F03AFF12208DF84000A8
:100A100002208DF841008DF842408DF8437010A8F7
:100A200002F048FF01224FF49061304600F0E8F8F0
:100A300001213046FFF740FF01213046FFF732FF2A
:100A400001212846FFF72EFF304600F06EF93046B0
:100A500000F09FF80028FAD1304600F075F93046D2
:100A600000F082F80028FAD1284600F05EF9284606
:100A700000F08FF80028FAD1284600F065F92846E2
:100A800000F072F80028FAD10121084603F00AFAB2
:100A9000154D284600F074FD684600F01CFE0F4816
:100AA00001A94C300090114881E811018020CDE966
:100AB00004404000069080000790202008904FF4EA
:100AC0004050CDE909046946284600F0E7FD0121C0
:100AD000284600F049FD12B0BDE8F0810024014035
:100AE00000280140002C014008000240C002002004
:100AF0000D4910B5884202D1012144150AE00B4985
:100B0000884202D10121041504E0094988420AD132
:100B10000121CC03204603F0F5F92046BDE8104042
:100B2000002103F0EFB910BD00240140002801406E
:100B3000003C01400029816802D041F4801101E0AD
:100B400021F48011816070470029816802D041F44E
:100B5000004101E021F4004181607047826822F485
:100B6000E0420A43826070470146002089684907D5
:100B700000D50120704710B50246002054680B0ACA
:100B8000C9B20C401168194202D0002C00D00120DB
:100B900010BD014600208968090700D50120704773
:100BA00038B501211C2003F0A1F9FF20ADF80000A9
:100BB00000248DF8034003258DF8025069460D4846
:100BC00001F0EAFA0120ADF800008DF803408DF83D
:100BD00002506946084801F0DFFA2320ADF8000012
:100BE0008DF803408DF802506946044801F0D4FAAC
:100BF00038BD000000080140000C01400010014019
:100C0000002A4268C9B201D00A4300E08A43426028
:100C10007047000010B542680E4B0C791A400B6803
:100C200042EA04221343436083680B4A1340D1E92C
:100C3000024222434C7943EA44031A438260C26A67
:100C4000097C22F47002491EC9B242EA0151C16214
:100C500010BD0000FFFEF0FFFDF7F1FF70B50724A7
:100C600009290AD9C568A1F10A0606EB4606B4406F
:100C7000A543B3401D43C56007E0056901EB41068C
:100C8000B440A543B3401D430561836BC3F30154D6
:100C9000121B921C02EB82041F22A2409343A1402C
:100CA0000B43836370BD826B491E22F4401242EAFB
:100CB00001518163704770B5072409290AD9C568B5
:100CC000A1F10A0606EB4606B440A543B3401D4316
:100CD000C56007E0056901EB4106B440A543B34098
:100CE0001D4305611F23072A09D2446B521E02EBE4
:100CF000820293409C4391400C43446370BD0D2A93
:100D000009D2046BD21F02EB820293409C439140B4
:100D10000C43046370BDC46A0D3A02EB8202934037
:100D20009C4391400C43C46270BD816841F008014E
:100D3000816070470029816802D041F4A00101E080
:100D400021F4A00181607047816841F00401816055
:100D5000704700210160017141718160C160012112
:100D60000174704770B51E4C214694F83800B1F8F4
:100D7000425006281ED9B4F84A10B4F84C00A1EB32
:100D8000000202F10902122A04D8FFF757FB0022E1
:100D9000144B0AE0884204D2FFF750FB0022124BAA
:100DA00003E0FFF74BFB0022104BFFF730FAFFF791
:100DB0008AFB09E005D12846FFF740FB0C4A0D4BA2
:100DC000F3E70D4951F82000C5EB45116063B0EB26
:100DD000410F03D9C5EB45104000606370BD0000B2
:100DE0006004002000003440000033400000354023
:100DF0006766666666E64B40208F000810B50C4CAF
:100E00002078400713D5FFF7ADFF0A49A08E088070
:100E100008483038018821F010010180001F018846
:100E200041F010010180207820F00400207010BDF6
:100E30006004002040040040F0B4184816494FF404
:100E40009677436C08468A68046815485FEAC25C76
:100E500042F00806007822F008054FEA047415D520
:100E6000002C08DB120714D408B1082811D1BB42AA
:100E70000FDA8E6007E012070BD508B1082808D1F9
:100E8000BB4206DA8D60F0BC05F05CBF002CF2DAE4
:100E9000E8E7F0BC70470000B002002048010020E5
:100EA0002B07002070B506464089204B204C4FF49C
:100EB0008071002580B362887AB1012A0CD1E18863
:100EC000491C89B2E1803289914205D36580E58071
:100ED000FF2801D0401E708170BD7088228890422A
:100EE00001D9012200E00022184601F0DEF97088E5
:100EF000B18801442088401C80B220808142EBD818
:100F00002580A088401C80B2A080F1888842E3D36D
:100F100001206080A58070BDFFE70022184601F027
:100F2000C4F9A580E58025806580F4E7000C0140C8
:100F3000D0050020FEE70000FCB505464FF6FF7621
:100F400000200C46ADF8006048F205078DF804005B
:100F500020E000BF15F8010B8DF8040001A9084638
:100F600002F0ECF8BDF800009DF8041080EA0120C2
:100F7000ADF800005FF00000BDF800100A0402D5D3
:100F800087EA410101E006EA4101401CADF800108A
:100F90000828F1DB641EDDD26946084602F0B8F885
:100FA000BDF80000FCBD00000246002004E000BFC8
:100FB00012F8013B1844C0B2491EF9D27047000034
:100FC00070B5144A85B01088002413490194009428
:100FD000039420460494138807E00D8B009E35444B
:100FE0000095CD8B019E3544019515889D42F4D026
:100FF000401CC0B28028EED30098411107484180C0
:10100000848001984111064881830183818205B063
:1010100070BD000034070020B0020020EA05002067
:10102000D804002030B50E4902880A800C4A438853
:10103000083A13800B1F808818802024151F2C80ED
:101040000020401C80B27328FBD341F211100880AD
:1010500044F64800108047F2480018802C8030BDCC
:10106000202C0140114944F648000880091D46F62D
:1010700048000880091D41F2111008800B48001F2C
:10108000018841F02001018009480021A0F8641086
:10109000A0F86210A0F86010A0F85E10A0F85C1034
:1010A000A0F85A100348418181827047182C0140F2
:1010B000B0020020640000202DE9F047494B4A4867
:1010C0000021DA7A0778802A27F0010676D31C6897
:1010D000464B02F01F0253F82220454B14421A6877
:1010E00002D042F0200201E022F02002DFF804A149
:1010F0001A60424CDFF8F8C09AF80050DFF8F89018
:10110000B4F904409CF846C0022D58D11D89C5F39E
:10111000C008C5F30025A84551D0354D303D95F8A0
:101120000280B8F1000F06D0B8F1010F0DD0B8F170
:10113000020F49D120E0110546D5910644D4012182
:10114000A97027F0040101703EE016053CD4960614
:101150003AD57E0738D446887EBB4480002C09DD12
:1011600047F0050101700221A9702549B1F844102A
:10117000018229E0A97027E0C7880FB9002C12DC92
:10118000077B67450FD11F4FBF895FEA47780AD4B5
:101190005FEA877807D45FEA427804D55FEA82681D
:1011A00001D5FF0710D006704180A9F800104181D9
:1011B0000182A970D9738AF8001005E00DE006706D
:1011C0004180A9F800104181C48080F80CC050090A
:1011D00060F3CB221A60BDE8F08706704180418140
:1011E000F9E70000F005002058090020809300086E
:1011F000B00200202B07002024010020EA05002077
:1012000048010020640A00202DE9F04796B0002430
:101210000C940D940E940F9472B69048816941F429
:1012200000718161816941F4806181614FF4004006
:1012300002F02EFE8A4D00212846FFF73DFB0021DB
:101240002846FFF72FFB874E00213046FFF72AFB89
:10125000854F0021384600F087F901204FF4704196
:10126000401C8842FCD32846FFF742FCB14630467A
:10127000FFF73EFC384600F083F94FF46020CDE9DB
:1012800012048DF8454001204FF004088DF8440009
:1012900010948DF8508010A92846FFF7BBFC01235D
:1012A0001A4605212846FFF706FD012302220621E2
:1012B0002846FFF700FD0123032207212846FFF7F8
:1012C000FAFC012304220F212846FFF7F4FC3846DC
:1012D00000F056F9684600F0FEF96148634E4C3064
:1012E0000090CDF80C80CDE901648020CDE9044068
:1012F0004000069080000790202008904FF4405056
:10130000CDE909046946384600F0C8F901212846AC
:10131000FFF7D2FA0121384600F026F901212846CC
:10132000FFF7C0FA47F2305115941598401C1590FC
:101330008842FAD301212846FFF7FCFCADF82C4087
:10134000A04640F2DC5A4FF4007420E05046CDF83D
:1013500054801599491C15918142FAD330880D9912
:1013600008440D9070880E9908440E90B0880F992B
:1013700008440F90F0880C9908440C9001212846ED
:10138000FFF7D8FCBDF82C00401CADF82C00BDF8D0
:101390002C00A042DAD30D98354A40F3CF163348DB
:1013A0000A3006830E9941F3CF1444830F9941F319
:1013B000CF1383830C9941F3CF1CA0F804C0ACF584
:1013C000C05C40F2C371ACF59B7C8C450ED2A6F597
:1013D000C856363E8E4209D2A4F5C854363C8C42DB
:1013E00004D2A3F5C853363B8B4203D3D18841F4D2
:1013F0008041D180D188490407D41E49028B21F84D
:101400005C2F428B4A80808B888000212846FFF722
:1014100053FA0021384600F0A7F800212846FFF7CC
:1014200041FA00214C464846FFF73CFA0220C1022F
:10143000401C8842FCD32846FFF75AFB2046FFF7A2
:1014400057FB384600F09CF8FFF740FA0A493C2069
:10145000087062B616B0BDE8F087000000100240C8
:101460000024014000280140080002403605002009
:10147000640A0020C40C00202807002070B5204B0F
:1014800040F6C81441F2B7055B6C48F6E6065C43CB
:1014900005EBA4341B4D73434EF6F61606EBA3334F
:1014A000C5E90443D460401A5361106091688842D2
:1014B00002DA4942884200DC116010684343107E22
:1014C0000341906A19189162506A814200DD90626E
:1014D000916A106A814201DB084600E09062A861CF
:1014E00011684C43117C0C4108412118B2F91C00D1
:1014F000884204DBB2F91A00884200DC08B270BDF1
:10150000480100202801002010B54FF40054204667
:1015100000F0ACF8002813D00A49087840F0080021
:101520000870204600F014F80021074800F01CF86D
:101530000648C17E012903D10021C176012101772E
:1015400010BD00008A06002044000240680B002005
:10155000C10002D5024908607047024948607047DF
:1015600004040240000002400029016802D041F05A
:10157000010102E04FF6FE72114001607047000069
:1015800001684FF6FE721140016000210160416068
:101590008160C1603149314A0839904203D14868BD
:1015A00040F00F0006E02D4A1432904204D1486802
:1015B00040F0F00048607047284A2832904203D13A
:1015C000486840F47060F5E7244A3C32904203D109
:1015D000486840F47040EDE7204A5032904203D111
:1015E000486840F47020E5E71C4A6432904203D119
:1015F000486840F47000DDE7184A7832904203D121
:10160000486840F07060D5E7154A111F904203D139
:10161000086840F00F0006E0114A1432904204D1ED
:10162000086840F0F000086070470D4A2832904288
:1016300003D1086840F47060F5E7094A3C329042F3
:1016400003D1086840F47040EDE7054A50329042FB
:10165000EAD1086840F47020E5E700000800024085
:1016600008040240406880B2704700000146002034
:10167000CA0001D5034A00E0034A12680A4200D0BA
:10168000012070470004024000000240002A026866
:1016900001D00A4300E08A430260704730B5036816
:1016A00047F6F07293430C6A8A682243D1E90445F5
:1016B0002C4322438C692243CC6922434C6A224347
:1016C0008C6A22431A430260CA6842600A688260D8
:1016D0004968C16030BD0021016041608160C16026
:1016E000016141618161C161016241628162704752
:1016F00010B5114C8CB000212046FFF735FF204675
:10170000FFF73EFF0D4800900D480021CDE9010193
:101710006420CDE903018020CDE9050107910891FE
:1017200009910A9169462046FFF7B8FF012120463A
:10173000FFF71AFF0CB010BD5800024004380140FA
:10174000C407002010B501218CB0084602F0AAFBA6
:101750001E4C00212046FFF707FF2046FFF710FF31
:101760001B4800901B48019000211020CDE9020188
:101770008020CDE9041006910791089109910A9102
:1017800069462046FFF78AFF012202212046FFF723
:101790007DFF01218DF82F1004208DF82D008DF88C
:1017A0002E100E208DF82C000BA802F083F80F20CD
:1017B0008DF82C000BA802F07DF801212046FFF7E0
:1017C000D3FEFFF795FF0CB010BD000044000240AF
:1017D0000438014060070020F0B540F6AA222A49EB
:1017E000C284838B0C88E31A9BB20F2B0DD309881C
:1017F0008183037E00213BB1244BB3F90A40244B83
:10180000062C03DA818429E08184F0BD214C247800
:10181000022C02D0002CF5D0F0BD1F4C40F68B27D7
:10182000656C1B4CA5F22D16BE42B4F9004017D2D0
:10183000418B491C89B241836429EDD364214183E2
:10184000B0F92410914201DA01EB22128284641C67
:1018500020B24FF4007118808842DDDB1980F0BDA2
:1018600041F29416B542FADBB0F92450002D02DDA6
:10187000A5EB221200E0002282844183641E20B284
:1018800018800028EADDF0BD340700206400002045
:101890005C0400202B0700204801002010B50446FE
:1018A000B0F9020043F6991148438113E06840F211
:1018B0006662504301EBA030E060B4F9001043F6DB
:1018C000991251438A13216940F26663594302EB2E
:1018D000A131216104F0A4FE6061A18840F6AB2231
:1018E00008444010A0F515415539E062914205D9F0
:1018F000A0F5F851FF39521C91421DD249F25451C2
:10190000884202DDA0F5204002E0A0F5F850FF3843
:10191000206300EB400040F34F002085B4F9241011
:101920004A42904201DA104602E0884200DD084651
:10193000E083228461848AE0A0F5FE42FF3A41F20E
:1019400055518A4214D8A2F6AA20206300EB400029
:1019500040F34F002085B4F924205142E1838842AE
:1019600001DA084602E0904200DD1046404250E0B5
:10197000A0F5D442AA3A8A4215D2A2F6AA20206340
:1019800000EB400040F34F012185B4F924004242AE
:10199000E2832084914201DA104602E0814200DCB9
:1019A0000846608453E0A0F5AA42543A41F25653E7
:1019B0009A4215D2A2F6AB20206300EB400040F320
:1019C0004F002085B4F924104A42904201DA1046B3
:1019D00002E0884200DD08464042E083218419E0AD
:1019E000A0F5804241F254539A4215D2A2F6AA20A1
:1019F000206300EB400040F34F002085B4F9241031
:101A0000E1834A42904201DA104602E0884200DD5A
:101A10000846208462841AE0A0F52852AB3A8A4234
:101A200015D2A2F6AA20206300EB400040F34F013C
:101A30002185B4F92400E08342422284914201DAF4
:101A4000104602E0814200DC08464042A9E7B4F9B2
:101A50001E0041420948B0F9000041438913E1806A
:101A6000B4F920104942414389132181B4F922106D
:101A7000494241438813608110BD00005C0400208E
:101A800001210176704770471548164A4FF480418E
:101A90000078042821D002F13C03D08A9B88C01A28
:101AA00000B22F2801DD001108E0002801DD002030
:101AB00007E00D4B984201DA184602E0402800DDAD
:101AC00040209389184400B2884203DC40F26661EA
:101AD000884200DA08469081704791817047000083
:101AE0002B070020D8040020C0FEFFFF38B54B486C
:101AF0004B4902880B889A1A92B20F2A71D309882F
:101B0000484C01804FF0FF01E2884FF47A7355048E
:101B10004FF4967002D51622009103E0950403D588
:101B200015220091014670E0D50402D514220091DF
:101B3000F8E7150502D513220091F3E7550502D504
:101B400012220091EEE7950502D511220091E9E7F6
:101B5000D50502D510220091E4E7150602D50F2223
:101B60000091DFE7550602D50E220091DAE79506CF
:101B700002D50D220091D5E7D50602D50C220091A1
:101B8000D0E7150702D50B220091CBE7550702D508
:101B90000A220091C6E7950702D509220091C1E704
:101BA000D20702D008220091BCE72289550702D54E
:101BB00007220091B6E7950702D506220091B1E70A
:101BC000D20702D005220091ACE7A27AD20702D058
:101BD00004220091A6E7A289D40603D5032200912E
:101BE000A0E719E0140702D5022200919AE75407F2
:101BF00003D4940701D4D20702D00122009191E7C7
:101C00000020034602460146009002F039FFBDE87D
:101C100038400248FFF746B938BD0000580A002096
:101C200034070020640A0020F0B5594859498288D9
:101C30000B889A1A92B29C2A64D3098881805649EB
:101C40000A880146002A0B7843F0020156D1164655
:101C5000524A1C0715680246127822F0020274D517
:101C60004F4C0746E4887F785FEA845C02D547F0F2
:101C7000010701E027F001074770A704477802D564
:101C800047F0020701E027F002074770670401D41C
:101C9000E70703D0477847F008074770640603D585
:101CA000447844F0040404E01C0603D4447824F08F
:101CB00004044470EC0450D4354C9A07247824F082
:101CC000100423D4324D42782F7A2D78012A45F022
:101CD000100514D0022A16D02D4C042AA47804F141
:101CE000010C0CF0FF0C13D0072A25D0032A23D0B7
:101CF000052A21D0062A1FD021F0100142E0B907A1
:101D000002E00570F0BD39070029FADB0470F0BD70
:101D1000FA0601D41A060AD50170022C04D280F802
:101D200002C0BCF1020FF2D341F080012AE021F0A1
:101D3000100101708670F0BD877A7F06F7D5032CFD
:101D400004D8017080F802C0F0BD0FE05107D8D56B
:101D50001906D6D443F0800114E002704178CB0715
:101D600001D18907F0D522F010010BE0E9040BD472
:101D70009907E9D4818AC82902D2491C8182E3E704
:101D800043F00A010170DFE702708682DCE70000A1
:101D90000C0700203407002036070020B002002086
:101DA000640A0020094944F648000880091D46F6E7
:101DB00048000880091D41F6CC4008800348001FF8
:101DC000018841F02001018070470000182C01407B
:101DD000084946F668000880091D0880091D41F27F
:101DE000555008800348001F018841F02001018000
:101DF00070470000182C014010B5C28800210AB1BC
:101E0000032206E002890AB1022202E0428912B1ED
:101E10000122027000E0017004784FF4804344F620
:101E2000206244B1012C06D0022C07D0032C01D132
:101E30004180818010BD4380828010BD41F23331EA
:101E4000418040F6B731F4E730B5B1F86A5000236D
:101E50001A240D22854202DCB1F9680030BD4D889C
:101E6000854202DBB1F9000030BD01EB82056D88CF
:101E7000854201DD144601E013DA134604EB030248
:101E80004FEA52029A42F0D101EB830231F823105B
:101E900054889288521A001B424301EB622000B220
:101EA00030BD31F9220030BD054920B1086940F04C
:101EB00080000861704703484860034848607047E5
:101EC0000020024023016745AB89EFCD06494FF45E
:101ED0007A70CA68D20705D0401E0004000CF8D101
:101EE000FF20704700207047002002400E4A032068
:101EF000A2F1500182F83E00002048810B4908867B
:101F0000C862C8830884488490620948016DB1F5AD
:101F1000206F01DBA3219162807A002802D0906AB1
:101F2000404290627047000064000020400500209D
:101F3000480100200449002048810881C862886265
:101F4000024988627047000064000020D408002025
:101F5000F0B53B4988894A89801A80B20F2866D338
:101F600088894881CA8937480B3A272A26D28A7835
:101F700022BB8268364B42F480728260324A354C12
:101F8000354D12785607314A0AD4344E36881680B9
:101F9000334A12881A80334A12882280324A09E072
:101FA000324E36881680324A12881A80314A128898
:101FB0002280314A12882A8001228A702F4B304DAC
:101FC00019469A7F0968802A32D302F01F0255F819
:101FD000222011422CD0826822F48012184E826096
:101FE000123614461215B778521C62F38617254A2A
:101FF000B77093F816C01778BCF1800F27F002066F
:1020000008D30CF01F0C55F82CC011EA0C0F01D1AD
:1020100047F0020616701A7E802A0DD302F01F02C6
:1020200055F82220114207D144F400218160F0BD0F
:10203000826842F48012D1E724F40021F6E7000020
:1020400028070020B002002048010020D004002012
:10205000D2040020D4040020D6040020C0040020B4
:10206000C2040020C4040020C6040020C8040020CC
:10207000CA040020CC040020CE040020F00500207B
:1020800080930008D804002070B520488189028917
:10209000891A89B20F292FD3818901811C4B1D48D0
:1020A00019465D7A06681C4C096846F00402802DCA
:1020B00007D305F01F0554F82550294201D126F019
:1020C000040202609A7B802A17D302F01F0254F8A0
:1020D0002220114211D1026822F002020260DA7A53
:1020E000802A0ED302F01F0254F82220114208D198
:1020F000016821F00801016070BD026842F002022F
:10210000ECE7016841F00801F5E70000280700202E
:10211000F0050020B002002080930008F0B51D4CAF
:102120001B4A4FF0010C94F83B5094F80AE0144617
:1021300092F83C3094F838402B43651CEEB2154DB4
:1021400095F83D700025BEF1FF0F0AD0BEF1000FDB
:1021500006D18B4213D155700C2C01D282F8386015
:10216000F0BD834202D182F801C0F5E78B42F7D17E
:102170005570B80709E000BF82F83850F0BD8342BF
:10218000FCD1F84382F801C080070028F4D0F0BDEC
:102190006004002048010020F0B5CA78002502F054
:1021A0000F03D20601D58A7813430A784FF00F0E39
:1021B00012F0FF0F4FF001021CD004680F8802FAE2
:1021C00005F63740B74211D14FEA850C0EFA0CF7ED
:1021D00024EA070703FA0CF43C43CF78282F02D0F7
:1021E000482F02D002E0466100E006616D1C082D18
:1021F000E4D304600C88FF2C1ED944685FF000060D
:1022000006F1080702FA07F50F882F40AF420FD1F9
:102210004FEA860C0EFA0CF7BC4303FA0CF73C436A
:10222000CF78282F00D14561CF78482F00D10561A4
:10223000761C082EE4D34460F0BD0000F0B5144CC9
:10224000002801DAE36900E06368420D120185B2FB
:10225000C0F301579540C0F30346032F05D0C202D7
:102260000AD50322B240934307E023F0706263680B
:1022700023F07063636002E0AB4343F0706201B12E
:102280002A43002801DAE261F0BD6260F0BD00007F
:10229000000001400246002092680A4200D001205E
:1022A000704741617047016170470AB10161704731
:1022B000416170470F4A104B92F838105B5C8342C3
:1022C00001D1012004E00D4B5B5C834203D100206F
:1022D00082F83A0070470A4B5B5C834201D181204F
:1022E000F6E7084B595C814201D18020F0E70320DA
:1022F000EEE7000048010020389800084A980008DE
:102300003E980008509800080A4810B501784FF030
:1023100000024C0708494FF0FF0389684FEA01713A
:1023200005D5002901DA827210BD837210BD002923
:10233000FBDBF8E748010020B0020020F0B5194EA1
:10234000194C0022E31CA6F1060CB75CA518ED7829
:10235000FF5C0D430F43BD421FD01CF80270FF5CB1
:102360000F43BD4219D015460023A618F6780E4338
:10237000C6545B1C1CF80220DBB2062BF5D3C178D7
:1023800081700179C17000214218491C15711CF837
:102390000550C9B20629F7D3F0BD521CD2B2032AA8
:1023A000D3D3F0BD128F00086004002010B50246A0
:1023B0000021064B06205C186478944200D1084640
:1023C000491CC9B20629F6D310BD000048010020FF
:1023D000214810B590F8671000222048012936D115
:1023E0001F49898899BB1F491E4B4C6C40F6B83178
:1023F000B3F876308C4227DD1B49097821BB90F871
:102400002711491CC9B280F82711C8291CD380F8AC
:1024100027210146D0F82C4191F82811A34203DD71
:10242000052908D2491C01E041B1491E80F8281154
:10243000C9B2052902D3012180F82611191B074CC6
:10244000303CA162C0F82C31B3F5FA6F03D280F8AA
:10245000262180F8282110BDC40C0020B0020020E5
:10246000EA050020480100202B0700204FF4C0425D
:10247000C260002181620E22028241F26202426148
:10248000082202834FF46042428381834FF07842F6
:10249000C0E9082140F6C41101807047B0F900106E
:1024A000B0F90220891A41604269037E4A431A4109
:1024B000836A13448362426A934200DD8262836AC4
:1024C000026A934200DA8262C268836A4A43017CEC
:1024D0000A410B41D118B0F91C208A4201DA10469A
:1024E0007047B0F91A008842FADC08B27047000061
:1024F00010B514481449B0F894200B889A1A92B277
:10250000B2F5437F1DD90988A0F89410B0F8921055
:1025100020F8601F002242860C480D4CC288828041
:10252000C180C38983812489891AA4B2C48181604E
:10253000E11A0161074A818AC182928A8282511A14
:10254000816110BD48010020340700208C0C002060
:10255000400500206400002009480A49B0F8B22074
:102560000B889A1A92B241F684639A4206D309887C
:1025700020F8B21F4188818000214180704700000F
:1025800048010020340700200D480178C90702D017
:102590000C49098801E04FF6FA71416609490120AA
:1025A0001039088007482438018841F00101018072
:1025B00004481838018821F0180101807047000094
:1025C00048010020240400400A49D1F8982012B1A3
:1025D000521EC1F8982031F8922F521C21F81A2966
:1025E0004A6A521C4A628A8F521C8A8701F8400C40
:1025F00070470000480100201CB52D4890F83B3082
:1026000090F83C20934252D000248DF8044053406F
:102610008DF800309DF800300122012B08D09DF884
:102620000030022B09D09DF80030042B0AD00DE0B9
:102630001F498DF80420443108E01D498DF804201D
:10264000463103E01A498DF8042048319DF80420F2
:10265000012A2CD190F83D309DF80040154AA34244
:1026600017D090F83E309DF80040234208D0B0F8D3
:102670004C30A0F84A300B881488E31AA0F84C308C
:1026800090F838302BB1B0F840301488E31AA0F835
:10269000423012880A80A0F8402010F83E1F9DF8B2
:1026A0000020114300F801199DF8001001701CBDB5
:1026B000600400203407002070B5344D40212846C6
:1026C000FFF7E8FD840080212846FFF7E3FD44EA98
:1026D0004004A9152846FFF7DDFD0443E1B22C4C68
:1026E00094F878508D4250D04D4084F87810012DE8
:1026F00003D0022D01D0042D47D194F87C00A843CB
:1027000084F87C0094F87B20AA420FD084F87B5098
:1027100094F87A2001238B401A4207D11A4384F897
:102720007A2094F87910491C84F8791094F879107B
:10273000042928D330B1012811D002280FD0042851
:102740000DD012E01348C18821F04001C1802078EB
:10275000002184F83B1020F06000207005E0217813
:1027600041F02001217084F83B000B4994F83B00B4
:1027700091F82720904204D081F8270007492020B3
:10278000087000F00DF884F8545070BD001001403E
:1027900048010020640A0020C40C00202807002003
:1027A00070B50D4D40212846FFF774FD840080214F
:1027B0002846FFF76FFD44EA4004A9152846FFF7B5
:1027C00069FD04430548072100F8784F0171002195
:1027D00041708170C17070BD00100140480100203F
:1027E00070B5344890F83A10CA43920761D001F0AE
:1027F000030280F8392090F83D305B061B0E80F80C
:102800003D30012A01D0812A02D15B1C80F83D3085
:102810000278D2074DD0DBB203F00102C3F34004CB
:10282000A24246D1B0F856400025641CA0F856409C
:10283000204CA0F8585090F83E60A47AB24202D0E2
:1028400080F83E200DE0A607B6EB837F02D080F82B
:102850003F5006E090F83F30642B02D25B1C80F8BA
:102860003F3090F84030642B0CD25B1CDBB280F818
:102870004030022B06D204F00103934202D102221F
:1028800080F84020012901D0002912D190F8382089
:10289000416E00EB820291610163D0E9061211449E
:1028A000D0E908231A441144826A1144C26A1144CF
:1028B000416370BD48010020FEE700002DE9F04FA4
:1028C00000BF00209E4E9F4AA6F51271A6F5BE7964
:1028D000A6F1440B06F1440E804601F5E074A1F127
:1028E000780301F5457A1D5C15F0C00706D0402F2E
:1028F00051D0C02F77D0802F76D004E115F01F057E
:1029000004D0154440F080072F7201E082F808805F
:10291000012826D0022824D0032822D0042820D041
:1029200008281ED010281CD0874D55F820C0DCF890
:10293000005054F820703D40CCF80050824D55F8BE
:1029400020C0DCF8005056F820703D43CCF8005011
:102950001D5CAD0659F820502F6813D53AF810C009
:102960003EE051F820502F6854F820C007EA0C07C9
:102970002F6051F820502F6856F820C047EA0C0706
:102980002F60E5E7DFF8B8C10CF1F00C5CF820C06F
:1029900007EA0C077EE015F01F0504D0154440F04F
:1029A00080072F7201E082F8088001281DD00228DC
:1029B0001BD0032819D0042817D0082815D01028B8
:1029C00013D0614D55F820502F6854F820C007EA05
:1029D0000C072F605C4D55F820502F685BF820C025
:1029E00047EA0C0756E00BE056E051F820502F68FC
:1029F00054F820C007EA0C072F6051F82050ECE78C
:102A000015F01F0505D0154440F0800785F82170AA
:102A100001E082F82180012825D0022823D0032854
:102A200021D004281FD008281DD010281BD0464DC7
:102A300055F820C0DCF8005054F820703D40CCF828
:102A40000050414D55F820C0DCF800505EF8207071
:102A50003D43CCF800501D5CAD0615D53A4D3AF813
:102A60001070CC3514E051F820502F6854F820C075
:102A700007EA0C072F6051F820502F685EF820C03D
:102A800047EA0C072F60E6E72D4D3AF81070E03D5D
:102A900055F820502F6036E015F01F0505D015447D
:102AA00040F0800785F8217001E082F8218001283C
:102AB00030D002282ED003282CD004282AD0082871
:102AC00028D0102826D0204D55F820C0DCF8005022
:102AD00054F820703D40CCF800501B4D55F820C0F4
:102AE000DCF80050164F883757F820703D43CCF87B
:102AF00000501D5CAD06B1D4114F3AF81050E03FC4
:102B000057F820703D60401CC0B21128FFF4EBAEB6
:102B1000BDE8F08F51F820502F6854F820C007EA24
:102B20000C072F6051F820502F68DFF814C00CF10B
:102B3000880C5CF820C047EA0C072F60D9E700003A
:102B40000C960008F0050020089400084FF4077167
:102B5000C1824FF45861018340F61451818370475C
:102B6000F0B5C48AB0F900608681B0F90250C58121
:102B7000B0F904300227002101220382AB4204DBBA
:102B8000B54202DDC78042810CE0B34204DBAE42B5
:102B900002DDC78041811CE09D4205DBB34203DDBD
:102BA000C2804781018115E0B54204DB9E4202DD0F
:102BB000C280418105E0AE4205DB9D4203DDC1805C
:102BC0004281078106E09E4204DBAB4202DDC18008
:102BD00047810281C388458900EB430700EB450527
:102BE000BB89AE899B1B0FFA83FEA0F812E0068911
:102BF000AB8900EB460CBCF80CC0A3EB0C03838242
:102C0000B0F91830B7F90CC0A3EB0C0CB4EB4C0FB7
:102C100004DA80F82010A3F1A10113E0A64503DD3A
:102C200080F82010B9890BE026B1012E04D0022EC5
:102C300010D004E0062100E0052180F82010A989C9
:102C4000091B6D31418309B2B1F5586F04DB5B1E7E
:102C5000438304E00421F0E7002900DC4283418B38
:102C60008183F0BD0B49002288760A62CA614A62FC
:102C7000094A32F9103002EB40028B62B2F90220AD
:102C8000CA62064A32F810000882A1F86000A1F872
:102C90006200704700020020629800085698000801
:102CA0002DE9F05FFE48FF4982880B889A1A92B29C
:102CB0000F2A44D30988FC4A818082461188012763
:102CC000FA48FB4D002479B3491E1180C473F94AB8
:102CD00084620168B2F902204E0742F6AA2318D492
:102CE000EE8846F40056EE80F24D2D78AD0709D5FA
:102CF000856825F080058560A0F87C4080F87E40DE
:102D000080F87F40CD0404D480F8F070C0F8EC4027
:102D100003E080F8F0404D0707D49A4205DB80F8C5
:102D2000F470A0F8F24004E010E080F8F4404D07A1
:102D300003D49A4201DBC90703D080F81141BDE8F2
:102D4000F09F80F81171A0F81241F8E78046B0F8C2
:102D5000181143F69820814202D2491CA8F8181194
:102D600001F0A4FED44EDFF838B396F85000ABF172
:102D7000180B10B1FEF7A0F905E09BF8001021F048
:102D800001018BF80010FFF723FB00F0EDF9CB48B1
:102D900041F268024FF40061406C904201DBC84A86
:102DA00004E0B0F57A6F02DAC54A121D1160B6462A
:102DB00096F85110DFF8F492DFF808C3C24EC90745
:102DC000A9F1300937D09CF80E1080292FD398F83C
:102DD000002092072BD498F80F2089F80520B54AD7
:102DE0004946137823F002031370ABF802409BF8B6
:102DF000003023F001038BF80030AA79520611D479
:102E00004A89B2F5FA7F03D2521CA9F80A2012E0CF
:102E100040F63C72904201DD00201CE1082089F858
:102E2000037018E1CC700020A9F80A4013E189F87A
:102E30000340A9F80A40D8F80800010501D5082088
:102E400009E173469EF83FE05FEACE714AD098F8F8
:102E50000F2089F805209CF8091080294DD398F897
:102E60000010490736D4E988890404D520F02000F1
:102E7000C8F8080036E0ABF802409BF8003040F09C
:102E8000200023F001038BF80030C8F808009CF8FC
:102E9000170080280BD300F07F034FF00040DCF8D0
:102EA0000010D840014202D188F8047001E088F88F
:102EB000044098F80400C00702D15FEA8E7005D57F
:102EC0000320032A01D089F80870C4E00020C8F864
:102ED0002840C0E020F02000C8F80800E88820F46E
:102EE0000050E88098F8260101280DD093F863007F
:102EF0001F4658B1FDF7A0FF13E0D8F8001041F0CD
:102F00000401C8F80010B1E70920A4E0D8F80800CF
:102F1000C10502D520F0080001E040F00800C8F823
:102F2000080098F846004FF4804198B101281DD060
:102F300002283078C0F3810029D08A1E012830D0C1
:102F400002282ED0A8F81411604890F85E000428DA
:102F50002AD01EE0307843F21E52C0F381000128CF
:102F600012D0022810D042F614600AE0307842F6FF
:102F7000CC42C0F38100012806D0022804D043F2DD
:102F8000EB10A8F8140104E0A8F8142101E0A8F857
:102F90001411A8F8441000BF97F87000012808D059
:102FA00016E0A8F81421CFE743F69910A8F84400DA
:102FB000F2E7307842F26662C0F3810001280ED059
:102FC00002280FD041F6E120A8F81401A8F8442007
:102FD0009BF80020D20708D0BBF8102007E0A8F823
:102FE0001421F3E74FF40050EEE732488288AAF844
:102FF000122010B2B8F944205043C0F38F32484633
:10300000A9F814208A4200D9818231490978C90679
:1030100005D5828A41F233318A4200D28182B8F8E2
:103020000810C1F3C002C1F300218A4205D1828A8F
:1030300041F699118A4200D98182A97AC90700D044
:103040008482B9F81400C8F8280000287FF7E4AE9D
:103050002048047002209AF81A1099B902284DD01D
:1030600080B116490B789E0608D5AE79760605D54F
:10307000174E3678F60966F386130B70E98821F44B
:103080000261E9800D49496C4E2932DBEB88190653
:103090002FD5B9F81260761CB6B2A9F812601BE001
:1030A000700900203407002036070020B0020020FD
:1030B000640A0020EA050020C40C0020480100201A
:1030C000100C0140F0050020D8040020640000200E
:1030D0000C07002048070020B6F5FA6F04D3A9F8C2
:1030E000124023F08001E98008490B7823F00203A5
:1030F0000B708AF81A0088F80F0020E6318F00293B
:10310000AFD143F698213187ABE70000EA050020F4
:1031100070B500230C8863F30F02012505FA03F64E
:10312000344206D0C3F10F0605FA06F1114361F3EC
:103130000F025B1C102BF1DB028070BD70B5002309
:103140000C7863F30702012505FA03F6344206D032
:10315000C3F1070605FA06F1114361F307025B1C90
:10316000082BF1DB027070BDF0B51F4890F8663097
:103170001E48012B816821F4006232D11C4BDE888D
:1031800074062ED41B4D0F054FF00004B5F9025004
:103190001ED4194A526C642A11DC40F638629542FA
:1031A0000DDAB2040BD4027852070ED4B0F8D42052
:1031B00040F6B835AA4203D2521CA0F8D420F0BD84
:1031C00041F4006181605C81F0BDA0F8D440F0BDA5
:1031D00041F2CD018D42FADD997AC907F7D18260BB
:1031E000F3E78260F0BD0000C40C0020B0020020B4
:1031F000640A0020EA050020480100200C490D481F
:103200004B88426C03B982645B1C9BB24B80FA2BE7
:103210000CD3836CD21AC2640020488040F6B830C8
:10322000824203DB0449012081F80D017047000050
:103230007009002048010020B0020020F0B5364D92
:10324000364F044695F83B0097F83B102378084327
:10325000EE1C6278834205D1E0781146FEF75EFFEE
:10326000207908E094F802C084450CD1E17810463A
:10327000FEF754FFE07905F82F0F2878805D68701D
:10328000287BE877F0BD82421DD161461846FEF7E3
:1032900045FF95F84E1095F83B00814207D1B97A69
:1032A00009B1A17900E0617985F82F101EE06978F5
:1032B000012901D0A17922E0617927E0297841F044
:1032C0000401297012E0E1788142DBD119466046A1
:1032D000FEF724FF95F84E1095F83B0081420AD185
:1032E000B97A09B1617ADFE7217ADDE715F82F1F96
:1032F000895D6970C5E76978012906D0617A85F82A
:103300002F10B97A0029F1D1D8E7217A85F82F104A
:10331000B97A0029EAD0D1E76004002048010020F2
:103320000B48017821F0020100F8381B002100F859
:10333000181941778177332181854185082141849E
:10334000012100F81F1C034880F839107047000065
:1033500060040020480100200D4900B50B4851F8D9
:10336000012F40F8032F8988818008480121093006
:10337000FEF7E4FF054802211330FEF7DFFF0348A4
:1033800004211D305DF804EBFEF7D8BF6004002077
:1033900048010020094944F648000880091D46F606
:1033A00048000880091D41F2111008800348001FE1
:1033B000018841F02001018070470000182C014075
:1033C0002DE9F047664C674B0025A0780126654A39
:1033D000103305287ED2DFE800F00313113E110000
:1033E000108820F0010010801D805F480580001FBC
:1033F0000580001F0580FFF7CDFFA670BDE8F087B0
:10340000594941F244401C390880574945F6580053
:1034100024390880091D47F25800088052492020AD
:10342000283908800020401CC0B27328FBD3FFF766
:10343000B1FF4C4984F85C502C3147F6906008800D
:103440004848143006801D80108840F0010010802C
:103450000220A070D2E700215FF0010004EB4102DE
:1034600004EB4003B2F85020B3F850309A4200D237
:103470000146401CC0B20628F0D33C48405C84F8AA
:103480003900FFF74DFF1D2000F0F3F900F076F84A
:10349000374E38484FF4807996F83B10012904D014
:1034A00002291BD0042930D047E040218046FEF796
:1034B000F1FE870080214046FEF7ECFE47EA400718
:1034C00049464046FEF7E6FE074347F0010084F810
:1034D0003B0000E03DE0224809302CE040218046DE
:1034E000FEF7D8FE870080214046FEF7D3FE47EA6C
:1034F000400749464046FEF7CDFE074347F002002D
:1035000084F83B001648133015E040218046FEF752
:10351000C1FE870080214046FEF7BCFE47EA400717
:1035200049464046FEF7B6FE074347F0040084F8DC
:103530003B000B481D3002F03BFF94F82F0086F84B
:1035400038001D2000F0ABF90420A0700A48057077
:1035500054E7108820F0010010801D80A5704DE711
:1035600060040020000800403C2C0140188F000837
:1035700048010020001001402B0700202DE9F041F8
:10358000344C14F82F0F344DE07240212846FEF7DA
:1035900081FE860080212846FEF77CFE46EA400632
:1035A000AF1539462846FEF775FE0643207BF1B27B
:1035B0002F3C814215D084F83C0040212846FEF77C
:1035C00069FE860080212846FEF764FE46EA400632
:1035D00039462846FEF75EFE064384F83B60FFF757
:1035E0000BF81E4D95F83B00012827D0022828D063
:1035F000042829D0174894F83B102730085C04F8B9
:10360000300F14F80109FEF7D1FE04F82F09A87A4B
:1036100000B10120607001F0E1FA94F84E0094F8D6
:103620003B10884206D094F83800062802D2401C8D
:1036300084F8380084F84E10BDE8F0810548093060
:1036400004E00448133001E002481D30BDE8F041B9
:10365000FFF7F4BD60040020001001404801002085
:103660002DE9F041524991F87200AA287ED191F8D3
:10367000730055287AD14F4C00200A5C2254401C1C
:10368000C0B27428F9D34C4E2069C6F80100A08A54
:10369000A6F80500D4F81600F060D4F81A003061DE
:1036A000D4F81E001234706102F028FE4349608A8B
:1036B000888102F03DFE207D123CC007307802D0A8
:1036C00040F0040001E020F004003D4930704FF468
:1036D00080403C4D886114F8280F85F82000608BED
:1036E0006880A08BA880E08BE880208C2881608C8B
:1036F000354F688194F8240087F8D20014F8011C33
:10370000304686F83B100026C0F89C60FFF724FE88
:103710002E48A18E0183E18E4183218F818394F80D
:103720004210283C012908D0022901D0032909D0E0
:10373000297821F00C01083107E0297821F00C01EB
:10374000091D02E0297841F00C01297094F86E20DF
:10375000012162B1012A01D0022A0BD087F846105C
:1037600094F864301A4A4BB1518108E014E087F8AC
:103770004660F5E7022287F84620F1E7568194F883
:10378000701001290AD094F86D1051B101290BD0A5
:103790004FF48051A0F87610BDE8F08144F21C711E
:1037A000F8E74FF40051F5E741F25551F2E7000018
:1037B00000FC0008C40C0020480100206400002028
:1037C0005C0C0020D8040020B0020020400500203E
:1037D000640A00207CB50121082000F087FB4FF42B
:1037E0008070ADF8040010248DF8074001208DF89A
:1037F000060001A91548FEF7CFFC0121092000F0C1
:1038000075FB01211248FEF719FD0820ADF80000F4
:1038100004208DF803000F4E03258DF802506946F1
:103820003046FEF7B9FC08213046FEF73AFDADF808
:1038300000408DF803408DF8025069463046FEF78F
:10384000ABFC10213046FEF72CFD7CBD001401407E
:1038500000023000000C0140FEE7704700F01F023C
:10386000012191404009800000F1E020C0F8801162
:10387000704700F01F02012191404009800000F1D3
:10388000E020C0F88011704700F01F020121914034
:103890004009800000F1E020C0F80011704700F0FE
:1038A0001F02012191404009800000F1E020C0F892
:1038B0000011704770B50F23C47801780122F4B16C
:1038C000144C2468457804F4E064C4F5E064240AE8
:1038D000C4F10406E3408478B5401C402C4301F158
:1038E000E021230181F80034007800F01F018A40B4
:1038F0004009800000F1E020C0F8002170BD01F017
:103900001F0082404809800000F1E020C0F88021BB
:1039100070BD00000CED00E0024908430249086058
:10392000704700000000FA050CED00E02DE9F05FA3
:1039300000261D20FFF792FF6C4CDFF8B4B1A4F114
:10394000B800A77E90F83810DFF8A8E1DFF8A8A14A
:1039500000258F427ED0E776A176626A036B5A43D8
:103960004FEA12499BF80820120702D51EF80120E1
:1039700000E00A4694F812C0BCF1010F09D004EB34
:103980004206B6F902C0C4F828C0B6F90460E6627F
:103990000CE043F6FF7CC4E90A5C90F83DC05FEAA6
:1039A000CC7C01D012B102E0052A00D1012600EB47
:1039B00047074FF0804CBF893F04B7FBF3F3E36147
:1039C000476BBCFBF7F7276294F813C0BCF1000FFC
:1039D00006D0BCF1010F05D03B4403EBD3735B1061
:1039E000636201E03B466762DFF810C14FF6FF7784
:1039F00007EA8307ACF808709AF8007090F80A801C
:103A000090F83DC0082F08F003070CF0030C05D018
:103A100067450BD1B8F1000F05D008E0674505D028
:103A2000B8F1000F03D05B42636200E06562C6B18B
:103A3000636A002B03D006DD228D05E00AE0304BDF
:103A400033F8122000E0A28DA4F86020227822F042
:103A5000200222709AF80020042A07D0082A05D0F4
:103A600012E0B4F8603003EB0902EDE780F8405053
:103A700065629BF80800000701D51EF80110204878
:103A800030F81100A4F860001E49606A09883E31D0
:103A90004843B4F8601001EB204006B21D20FFF748
:103AA000F3FE606A002807D021784FEA81600ADDC2
:103AB000002804DAA08D09E0B4F8600006E0E06AAE
:103AC000B04208DB0CE0002802DA208D208208E0FA
:103AD000A06AB04204DD208241F02000207000E0A6
:103AE0002682257565752586BDE8F09F00020020B9
:103AF000B0020020449800082B0700203C0A002058
:103B0000569800082404004043184FF48042934222
:103B100010DD904202DD104600210BE0914202DDF3
:103B20000020114606E08003B0FBF3F000B2C0F5C0
:103B3000804109B241EA00407047F0B541F2862366
:103B40000022C3600E24826204824CF2E82508261B
:103B50004561068343F6FF774283878340F2492E0F
:103B60004FEA873CC0F808E0C0E9082CCB608A62C5
:103B70000C824D610E834A838F83B4208860C1E933
:103B8000082CF0BD002181620949C1600E2101822B
:103B90004FF6BF514161082101834FF440414183F9
:103BA00043F6FF7181830907016202494162704750
:103BB000638A010000C0FF0F064941F6A260088039
:103BC00005480168054A01F4E06111430160BFF353
:103BD0004F8FFEE7442C01400CED00E00400FA0595
:103BE00038B501210D2000F081F94FF4E060ADF807
:103BF000000018248DF8034003258DF80250694613
:103C00000D48FEF7C9FA4FF46040ADF800008DF89A
:103C100003400A4C8DF8025069462046FEF7BCFA74
:103C2000A014ADF8000048208DF803006946204636
:103C3000FEF7B2FA38BD000000080140000C014058
:103C40002DE9F0410121CE028CB0304600F04EF952
:103C5000DFF86C81404601F037FC08A801F060FEF7
:103C60004FF45860ADF824000024ADF82040202027
:103C7000ADF822000125ADF826408DF8285008A99E
:103C8000404601F0FFFD0021404601F052FE4FF694
:103C9000FF71404601F057FE01220021404601F02D
:103CA000E3FD0121404601F0CBFB04A801F0E3FB5A
:103CB000ADF81060A802ADF81200ADF81440A220D3
:103CC000ADF816002803ADF81800ADF81A40ADF8AD
:103CD0001C4004A9404601F0BDFB6027ADF8007010
:103CE000ADF80440ADF80840ADF80C40ADF8024026
:103CF000ADF80640ADF80A40ADF80E4069464046C2
:103D000001F0A2FC6946404601F0E4FC69464046E9
:103D100001F02AFDADF8045040F61450ADF80070E3
:103D2000ADF80600ADF80840ADF80C40ADF8025013
:103D3000ADF80A40ADF80E406946404601F058FD26
:103D40000121404601F0A0FB0821404601F0BCFCE7
:103D50003146404601F0FEFC0821404601F042FD9C
:103D60003146404601F076FD7021404601F07FFD6E
:103D700018208DF82C008DF82D408DF82E408DF8F0
:103D80002F500BA8FFF796FD0D480C30018841F02D
:103D9000800101800A481430018841F0010101804E
:103DA000001F04800121404601F078FB8DF8285067
:103DB0000121404601F07CFB0CB0BDE8F081000021
:103DC000002C0140704740F213414160082181609E
:103DD0008621C1604FF48041016149424161002167
:103DE0000162C162704701627047000010B501882E
:103DF0004288891A09B20183B1F5005F02DBA1F59F
:103E0000804104E011F5005F02DC01F5804101838F
:103E1000B0F9182041685143C1618368846A5343F3
:103E2000C2681B12624303EB2222036A1A44114444
:103E300002628A13426241698A4203DB01698A4253
:103E400000DC11468A1AC0E90A21028E4FF403737E
:103E5000594302EBA13202860B4A1278082A04D198
:103E60000A4A936F03EBA1319167B0F93010B1F5B5
:103E7000804F02DDA1F5804103E0002902DA01F55F
:103E80008041018610BD00002B070020780A002029
:103E9000034A516821F440410143516070470000DA
:103EA00000100240044A0029516901D0014300E09A
:103EB000814351617047000000100240044A00290C
:103EC000D16901D0014300E08143D1617047000016
:103ED00000100240044A0029116901D0014300E0AA
:103EE000814311617047000000100240044A00291C
:103EF000916901D0014300E0814391617047000066
:103F000000100240044A0029D16801D0014300E0BA
:103F10008143D160704700000010024030B5244951
:103F20004A6812F00C03234A03D0042B01D0082B5B
:103F300026D002604A680F231F4C03EA1212A35CCA
:103F40000268DA4042604B68072505EA1323E35C08
:103F500022FA03F383604B6805EAD323E35CDA407B
:103F6000C2604B68032403F4404104EA933303EB3B
:103F70009161114B1B1F595CB2FBF1F1016130BD26
:103F80004A680E4B1A404B68140103F4803303D582
:103F9000C2F38342113202E0022404EB924213B1D5
:103FA0004B689B0301D5064B00E0024B5A43C0E728
:103FB0000010024000127A000400002000003C08BB
:103FC00000093D002DE9F041274CA615402120466F
:103FD000FEF760F9850080212046FEF75BF945EA8F
:103FE000400531462046FEF755F90543EDB2402124
:103FF0002046FEF74FF9870080212046FEF74AF958
:1040000047EA400731462046FEF744F90743F8B235
:10401000A842DBD140212046FEF73CF987008021F1
:104020002046FEF737F947EA400731462046FEF7BB
:1040300031F90743F8B2A842C8D140212046FEF723
:1040400029F9870080212046FEF724F947EA400736
:1040500031462046FEF71EF90743F8B2A842B5D113
:104060002846BDE8F08100000010014010B502684C
:10407000416802FB02F301FB01330D4CA34211D94D
:104080001B0E0E3B0B4C9BB212B234F8133009B22C
:104090005A43594342F38F3241F38F31C0E9022131
:1040A000012102E0C0E902210021017410BD0000DD
:1040B000E10BBF0E688C00082DE9F05FF848F94964
:1040C00002880B889A1A92B20F2A7DD30988018040
:1040D000F54802468189D2884B0703D48B0701D467
:1040E000CB0702D042F4007201E022F40072C280D9
:1040F0008246080702D45046C90604D5BAF806100D
:1041000041F0010102E0C18821F00101AAF8061086
:10411000E548FDF771FEE548B0F93A10B1F5804F7A
:1041200002DA491C418703E0E0494FF480404887A8
:10413000DFF87C9341F6CC40DE49D9F8502082422A
:1041400003DD886820F010008860DB48DB4F002525
:10415000038823B15B1E0380CD733D7027E0BAF85E
:10416000060044041BD4BAF80C30DC0617D41B0735
:1041700015D4030613D4830611D403050FD44306C4
:1041800003D5CF4B1B781B0609D5430707D4C305BE
:1041900005D4030703D4830401D4C00607D5C94856
:1041A000CD73C94B3D70C5831D8080F82A508B4666
:1041B0000846C98FC54CDFF818C351B1491EC187E5
:1041C000237823F0020300E0F4E023708BF80F5013
:1041D0000AE0217841F0020121703878012804D1E9
:1041E0009CF80000062800D13D703878DFF8E4E242
:1041F000B94E4FF001080A2877D2DFE800F0FDDB66
:1042000005DBFCFBDB76FAF902F08EF9A94890F8A1
:104210000D0108B9FEF7F2FFDFF898A2CB46AAF12C
:10422000300ABAF81810491C8AB2AAF81820D9F82E
:10423000440040F62821884202DAAAF8185014E017
:104240009A4940F6CC43C96899420EDBB4F9041090
:1042500043F69913994208DBB2F5FA7F05D3327819
:104260001AB9AAF8185086F800809C4A118869B1DA
:104270009AF804305B1CDBB28AF80430022B05D3B9
:1042800097498AF804500B885B1C0B80894CE17BB2
:10429000092912D002297CD0A4F83051B4F840107A
:1042A000A946C9B141F288354946AAF81890A842F2
:1042B00020DA3078012819D01CE079484430FEF724
:1042C000D5F8FDF713FEDBF84410CAF82C1041F2C4
:1042D0007C51CAF81C1060E2B08A2086F06A7063D4
:1042E000B06A3063A4F8408036E0A1E17C483170C8
:1042F000018011807B4890F8682040F63A20012A1E
:104300000DD0C4F8D81084F8EA10CAF82410B4F913
:10431000301001F21D52824218D8102317E094F891
:10432000282102B97049C4F8D81084F8EA80B4F999
:10433000301001F21D528242B4F8D80000B202D807
:1043400010231A4605E02023022202E02023102237
:10435000002000F0A1FB2086624864494FF492736C
:1043600090F86800012815D0DBF8440040F2DC52D8
:10437000904203DAB6F90A209A4215DBB4F84020DD
:1043800040F6C413521C92B2A4F840209A420BD2B9
:1043900012E01AE0DBF8442040F2DC50824209DAF5
:1043A000B6F90A00984205DA87F8009084F8EA9096
:1043B000A1F81A90BDE8F09F3C4AD268002AF9DCC7
:1043C00042F6E0629042EFDAF4E7B4F8301140F6DA
:1043D000B832914207D2324B183B1B78DB0702D12F
:1043E000491CA4F830118BB240F2DC518B4204E03E
:1043F000B8E096E0DDE0D8E0E0E002D842F6CC415B
:1044000003E0A4F8302143F26661F167CAF82C009A
:104410008AF80780364FA4F8405084F8EA50797F34
:104420005646D1B1F87F70B3208DB4F9301000B288
:104430000A23052200F030FB2086FD7787F81D5007
:10444000B4F91601B4F91411884257DA254991F8E4
:104450004D1019B300F1020052E000B2254901F0FD
:1044600013FDA4F8E400A16A814200DA08461D4960
:1044700000B2F08291F84D100029B4F9301003D049
:104480003623052203E005E040F24713362200F010
:1044900003FB01E040F266602086D1E72CE00000DB
:1044A0007009002034070020640A00204005002025
:1044B00048010020B0020020380700202B07002010
:1044C0000C070020040900201E000020EA0500203F
:1044D0002C0700206802002064000020200000203B
:1044E00022000020C40C00209AF9FFFFE4090020FC
:1044F0008C0C00205A8E0008083001E003DD801E7D
:10450000A4F8160101E0A4F81611B4F930104FF424
:104510008040814201DD20864CE70029FCDA2586B7
:1045200048E7D34ADBF8DC105846914202D2491CD6
:10453000C0F8DC10C17B082903D1D0F8DC1091420F
:104540000CD33D708168CA0502D521F0080101E055
:1045500041F008018160CBF8DC502BE7BDE8F05F4B
:1045600002F004BD9BF80F005E46092803D0358693
:104570008BF80F5050E1BF4C206A401C206202288B
:1045800009DDA08D012301B2A08B052200B200F04D
:1045900083FA2562E062B848A18D0180B9F8441021
:1045A0004180FDF77BFF308604E7BDE8F05F04F053
:1045B0001DBA9EF8000009287DD0FBE68BF80D514E
:1045C0009BF8281161B142F31100CBF8D850AB49E8
:1045D0008203F06280108A628103B062A84881621F
:1045E000A4480583D9F8441041F28830814207DAA3
:1045F0003078012804D1A34835700580A248058091
:10460000A24AA34B1088401C81B2A2481180C8293D
:1046100002D30478012C17D0B1F57A7F02D3047845
:10462000022C11D0B1F5FA6F02D3017803290BD017
:104630009BF80F00801E082877D2DFE800F010B04A
:10464000F1EF047677A2B5E605701580BAF806108A
:1046500021F40061AAF8061083F80080E8E7FDF76E
:1046600053FE99F800004C46400612D58A488078DF
:1046700004280ED0616C204682290ADA817A94F8E7
:104680003D0001F0030100F00300814201D001F080
:10469000FBFD3878062887D084F83F50206D774995
:1046A00040F311008203F06280108A628103B062DD
:1046B0007348816200E0AFE0FDF718FC6D485E468C
:1046C00080F80780BBF81401ABF81601606CABF8FA
:1046D0008250B0F5437F12DD4FF48040A6F8800091
:1046E000B06840F48060B06094F838100529AAD111
:1046F00040F01000CBF808008CE038705AE64FF418
:104700008041A6F88010B16821F48061B16040F268
:104710008A21884204DA2078400601D402F012FB94
:10472000B06840F01000B06074E098E0D9F8440040
:10473000B0F5437F07DA9CF80010062903D000BFCC
:104740008CF8005083E05548017821F04001017059
:10475000FDF7CCFB43F6FE70ABF816010BF1DC0461
:10476000FDF7D2FD4E4810F8341F21F00101017011
:10477000434925608D6241498D6208213970456445
:1047800018E63D48FDF772FEFDF7B0FB3948D9F851
:104790004410C16241F27C51C1610920ADE79AF831
:1047A0000600C006AAD4D9F844004C46B0F57A7F7A
:1047B00032DDFDF7A9FD2078400611D53648807816
:1047C00004280DD0606C82280ADAA07A94F83D1093
:1047D00000F0030001F00301884201D001F054FD14
:1047E00084F83F50B4F85000ABF8300001B24FF4F9
:1047F00080405D46814200DD2886FDF777FBA86892
:1048000040F48060A86094F838100529B8D140F0D1
:104810001000A860022070E73D70CBE513E0FFE7D1
:10482000D9F84400B0F5437F03DA9CF8001006295C
:1048300086D1BAF8061021F02001AAF80610FDF77B
:1048400063FD042059E79CF80000062802D087F891
:104850000080AFE509208EF8000005204DE70E48E6
:1048600085708CF8005086F85E50ABF83050A1E5AA
:10487000C0D4010080020020B4090020D408002028
:10488000A4080020220000202000002016000020A4
:104890001400002015000020600400203A070020CA
:1048A000780A002030B585B001210420FFF71EFBF7
:1048B0004FF40040ADF8100048208DF8130004A913
:1048C0001848FDF769FC01210846FFF7F7FA40F6A2
:1048D0008C20ADF8040003240020ADF80040ADF8B2
:1048E0000200ADF806004FF080456946284600F00A
:1048F000C9FF1C208DF80C008DF80D408DF80E407E
:1049000001208DF80F0003A8FEF7D4FF0122114605
:10491000284600F091FE0121284600F0BFFD05B0B9
:1049200030BD000000080140704700002DE9F04153
:10493000304CE07800285AD12078002857D0401E0B
:1049400010F0FF00207052D14FF49670208272B6A2
:10495000294F45F2AA50A7F872000020FDF7A4FAEB
:10496000264D13202860FDF7B1FAA8BB3420E8607B
:1049700002202861224E6E61286940F040002861C3
:10498000FDF7A4FA40BB00211E4A08465FEA255302
:1049900012F800C0BCF1FF0F00D00121401C80B212
:1049A0009842F5D3C1B9C4E9067639260127A06932
:1049B00010F8011B10F8012BA061E06901EB022146
:1049C00002886A612F6120F8021BE061FDF77EFA20
:1049D00010B9761EB6B2EAD20120FDF765FA62B6CA
:1049E00001F0A6FC0848816821F480418160BDE89F
:1049F000F081000028070020C40C002000200240A5
:104A000000FC000800FC0008B00200201948016802
:104A100041F010010160016821F0030101600168AB
:104A200041F0020101601448416841604168416001
:104A3000416841F480614160416821F47C1141602A
:104A400041680E4A11434160016841F08071016084
:104A500001688901FCD5416821F00301416041688A
:104A600041F0020141604168C1F381010229FAD19C
:104A7000704700000020024000100240000028089B
:104A800030B5044C039D6080A180E2802381658164
:104A900030BD0000580A00200A44824201DA10B2F8
:104AA0007047C91A8142FBDD08B270472DE9F04317
:104AB0004348DFF81081DFF81091C17F457A046820
:104AC00001260023414A424880292BD301F01F01CF
:104AD00058F821100C420146096802D041F4805177
:104AE00001E021F480510160CF0417D48F0415D563
:104AF000977AFF0707D0538199F800C02CF0020C79
:104B000089F800C00AE090F84670BFB14FF0020C7F
:104B1000012F18D080F8463080F81AC10F0B67F3C8
:104B20004D310160802D2AD305F01F0158F8211066
:104B30000C4201680CD041F004010BE080F84660A3
:104B400080F81A31EAE780F846C080F81A61E5E794
:104B500021F0040101604C070DD44C050BD5947A6B
:104B6000E40708D0538199F8005025F0020589F830
:104B70000050C0F898308C0864F38A210160917A63
:104B8000C90717D1134991F86410012912D11249AC
:104B9000496C32290CDC0178490709D501890905DE
:104BA00006D4D0F8981047F23054A14204D9568167
:104BB000C0F89830BDE8F083491CC0F89810F9E7B8
:104BC000F005002080930008EA050020640A002018
:104BD000B0020020C40C00204801002010B5FCF7F2
:104BE000C1F80F48018821F0020101800C491831F9
:104BF00009880C4A928E1144094A343211800849BE
:104C00000C390A8842F001020A80011D0A884FF619
:104C1000ED531A400A80018841F01201018010BD55
:104C20000C0400406004002006484188491C89B2F9
:104C30004180B1F57A7F04D38188491C81800021AD
:104C4000418070474C0700200F4810B5016841F0C3
:104C50000101016041680D4A1140416001680C4A40
:104C600011400160016821F480210160416821F454
:104C7000FE0141604FF41F018160FFF7C7FE054947
:104C80004FF00060086010BD001002400000FFF807
:104C9000FFFFF6FE08ED00E02DE9F0413149324D0D
:104CA0000888401C088028884FF00004000629D599
:104CB000FCF7D8F92D4A2E4807231778C8262D4926
:104CC000012F22D02C4FB7F806C0BCF1000F3ED008
:104CD000B0F80CC04CF0080CA0F80CC0B0F806C03E
:104CE0002CF4006CA0F806C0886820F004008860EE
:104CF000FC801370CE8700204FF49661401C80B278
:104D00008842FBD32C80BDE8F0811C4F97F800C08F
:104D1000BCF1010F0FD0BCF1020F11D0B0F806C0EA
:104D20004CF4006CA0F806C0886840F0040088606D
:104D300005203870DDE7B0F80CC04CF0080C03E03B
:104D4000B0F80CC04CF0100CA0F80CC0F0E70C4F01
:104D50003C70C78847F40067C780886840F004004B
:104D60008860C6E74C070020102C01402B0700206C
:104D7000640A0020B0020020700900202C070020E7
:104D800049070020704700002DE9F0434FF08040B4
:104D9000018A21F001010182AB48007800287CD112
:104DA000AA4FF87B002878D1A948406C322874DCDF
:104DB000A8488068DFF8A0924104A84DB9F8040023
:104DC0004FF0000403D4401CA9F8040026E1002899
:104DD00074D02978012611B1012912D015E1494674
:104DE000B0F5BE7FFAD92E70CC718C71EC702C723C
:104DF000287A0A18401CC0B2147228720F28F7D300
:104E000003E1B9F802204946824201D9EE7100E07F
:104E1000EC7191488A7908300F2A15D2CB79082B8A
:104E20000BD2C3F10708EB7912F800C003FA08F3BC
:104E300063441354CA79521CCA71CA79082A03D12F
:104E40008A79521C8A71CC7199F80610C8460F29CC
:104E500073D10D21FCF770F8A881010A6970C0B206
:104E6000A87088F8064098F816208A4265D198F80C
:104E70001510814261D198F80BC0794903230222B1
:104E80007848BCF1000F10D0BCF1010F02D0BCF18A
:104E9000020F14D080F86A2000E0C9E091F800C049
:104EA0002CF00C0C0CF1080C0FE080F86A6091F803
:104EB00000C02CF00C0C0CF1040C06E0A7E080F80C
:104EC0006A3091F800C04CF00C0C81F800C098F8E2
:104ED0000C10B6EB111F04D180F86E4087F84640E5
:104EE0000EE0B2EB111F04D180F86E6087F84660C7
:104EF00006E0B3EB111F03D180F86E2087F846203F
:104F00000B0717D001F00F01012901D0022915D09C
:104F100080F86C602C7198F80D102A7906FA02F36B
:104F20000B406B71082A41D2DFE802F00B0F4016EC
:104F3000212C333A80F86C40ECE766E080F86C2076
:104F4000E8E713B380F8704030E013B180F85060A8
:104F50002CE080F8504029E023B180F8656087F8A4
:104F6000036123E080F8654087F803411EE023B128
:104F700087F8F54080F84D4018E087F8F56080F834
:104F80004D6013E013B180F868600FE080F868406E
:104F90000CE013B180F8666008E080F8664005E038
:104FA00013B180F8676001E080F86740521CD2B20C
:104FB0002A71082AB1D398F80E102B4A8B0705D511
:104FC00087F8F16080F86460568104E087F8F1406A
:104FD00080F864405481C90702D080F8294001E07C
:104FE00080F8296098F8111000F86D1FC2781F48EA
:104FF000012A1FD009B3012922D04FF4805100BFEC
:10500000A0F876101A493C200870A9F80240A9F8C7
:105010000440B9F80210491CA9F80210B9F80210AE
:10502000B1F5FA7F04D940F2F511A9F802102C70FD
:10503000BDE8F08344F21C71E2E74FF40051DFE772
:1050400041F25551DCE700002B070020B0020020A0
:105050004801002000100140AC0C0020C4060020D4
:10506000D8040020C40C0020640A00204005002061
:10507000280700202DE9F05FFDF746F98E4D2888BE
:10508000A5F10406C0070AD0308820F0080030805F
:10509000288820F00900288001F054FED9E02888F3
:1050A000DFF81892DFF81882864C80071AD5B9F815
:1050B000001041F00101A9F80010B8F80000804983
:1050C00014315030088028884FF6F9510840288064
:1050D000308840F004003080FEF774FF84F83C0014
:1050E000BDE8F09F2888784F4007288871D520F0C8
:1050F00004002880FEF766FF94F83C108142EFD14F
:10510000308820F004003080FDF7D6FA2078410680
:1051100005D594F8541094F83B209142E0D03978AA
:10512000400621F00201397004D5FEF727FA97F8FE
:105130002F7004E094F83C00FDF738F90746DFF8DB
:1051400080B140F68C2A0BF1180B062F47D294F849
:105150003800B8423ED03846FDF7ACF82078C0079A
:1051600016D094F83A0094F8391000F003029142F6
:1051700006D0A17A00F0010001F00101884215D1AA
:10518000FDF702FAFBF73AFEFDF72AFB384689E005
:10519000FDF7FAF9FBF732FEFDF722FB3846FDF783
:1051A00013FA207840F00100207099E7288820F059
:1051B00008002880206B810801EBD000504515D2F3
:1051C000B8F800100844ABF80000308840F0080040
:1051D00003E00DE0308820F00800308080E7B9F867
:1051E000001041F00101A9F80010DFE75046E7E7A1
:1051F0000007288831D520F008002880308820F06A
:1052000008003080FEF7DEFE84F83C00FDF754FA1B
:10521000387820F0020038702078400604D5FEF778
:10522000ADF997F82F5004E094F83C00FDF7BEF874
:105230000546062D08D294F83800A842B5D0FDF7EF
:10524000A3F9FBF7DBFD2AE02048C18841F04001CB
:10525000C180BDE8F05FFDF7A3BAC006288825D558
:1052600020F010002880308820F01000308097F85F
:1052700038000C2802D2401C87F83800387840F0FB
:1052800002003870FEF77AF997F82F50787884F892
:10529000390094F83800A84287D0FDF775F9FDF77A
:1052A0009FFA2846BDE8F05FFDF78EB94EF2BE11B9
:1052B0000840288014E7000010040040000400406B
:1052C000240400404801002060040020640A0020FB
:1052D0002DE9F04F514F85B0388820F0010038801B
:1052E0004E480026103006804D4CDFF838A14FF0B4
:1052F000010894F85C0042F63029C10774D072B6F8
:105300004948816941F400718161816941F480619A
:1053100081614FF40040FEF7BBFD444D002128465B
:10532000FBF7CAFA00212846FBF7BCFADFF800B108
:1053300000215846FBF7B6FA00213E48FCF714F965
:105340002846FBF7D5FB5846FBF7D2FB4FF460200D
:10535000CDE902068DF8056000968DF810808DF875
:10536000048069462846FBF755FC01231A460F21A5
:105370002846FBF7A0FC01212846FBF793FA002002
:105380004946401C80B28842FBD328462E6001214A
:10539000FBF7D0FC28688007FCD524484C30006817
:1053A00094F85C1021F001012144A1F85000FBF7B2
:1053B0008DFA62B6FDF7EEFF47F69061AAF800108D
:1053C00094F85C00401CC0B284F85C000C2822D227
:1053D00012491431A1F80080388840F0010038806B
:1053E00005B0BDE8F08FFFE7134920F00100085A2F
:1053F00012490880114945F65800083908800F48BD
:1054000047F25801001F01800C4920200C39088008
:10541000AAF80090D4E70320A070E1E7000800405C
:10542000600400202C0800400010024000240140CD
:1054300000280140080002403C8F0008202C014059
:105440000029018802D041F0800101E021F08001B3
:105450000180704710B50A884B88CC881A438B8826
:1054600023431A430B891A434B8989891A430A43F8
:10547000A0F8442010BD0021018041808180C180BE
:1054800001814181818170470029818802D041F0EA
:10549000010101E021F001018180704700290188AC
:1054A00002D041F0010101E021F0010101807047CB
:1054B000002930F8441F02D041F4004101E0C1F35B
:1054C0000E010180704700004B4910B5884202D19F
:1054D0000121C41486E0B0F1804F09D047498842C9
:1054E0000DD101210220FEF7F5FC0021022064E02D
:1054F00001210846FEF7EEFC002101205DE0404955
:10550000884206D101210420FEF7E4FC002104209A
:1055100053E03C49884206D101210820FEF7DAFC1D
:105520000021082049E03849884206D10121102095
:10553000FEF7D0FC002110203FE03449884206D11C
:1055400001212020FEF7C6FC0021202035E0304953
:10555000884202D10121441444E02E49884202D1FC
:105560000121CC043EE02C49884202D101210C05E6
:1055700038E02A49884202D101214C0532E028490D
:10558000884206D101214020FEF7A4FC00214020E2
:1055900013E02449884206D101218020FEF79AFCBD
:1055A0000021802009E0204988420AD18415012188
:1055B0002046FEF78FFC00212046BDE81040FEF794
:1055C00089BC1A49884202D101210C040AE0184919
:1055D000884202D101214C0404E0164988420AD1D4
:1055E00001218C042046FEF78DFC2046BDE81040CA
:1055F0000021FEF787BC10BD002C014000040040D4
:1056000000080040000C0040001000400014004062
:1056100000340140004C0140005001400054014062
:1056200000180040001C00400020004000400140E5
:105630000044014000480140002A828901D00A4309
:1056400000E08A438281704730B5028C22F001026B
:105650000284028C8388048B22F0020224F07305FA
:105660000C882C430D8915434A882A43114DA842C2
:105670000BD0114DA84208D0104DA84205D0104DB6
:10568000A84202D00F4DA8420DD122F008054A8948
:1056900023F440732A4322F004058A882A438D8923
:1056A0001D43CB892B4383800483C9888186028470
:1056B00030BD0000002C014000340140004001409A
:1056C0000044014000480140028B22F008020A43D6
:1056D0000283704770B5028C22F010020284028CA3
:1056E0008488038B0D8823F4E6464FF6FF7303EAA4
:1056F000052535430E8922F0200203EA06161643DB
:105700004A8803EA02123243104EB04202D0104ED1
:10571000B04215D122F080064A8924F4406403EA9D
:105720000212324322F040068A8803EA0212324310
:105730008E8903EA86062643CC8903EA840434432F
:1057400084800583C9880187028470BD002C0140D4
:1057500000340140028B4FF6FF7322F4006203EA2B
:10576000012111430183704770B5028C22F48072CD
:105770000284028C8488838B0D8823F073031D437D
:1057800022F400730E894FF6FF7202EA06261E43CA
:105790004B8802EA03233343104EB04202D0104E2E
:1057A000B04215D123F400664B8924F4405402EA38
:1057B0000323334323F480668B8802EA03233343B5
:1057C0008E8902EA06162643CC8902EA0414344381
:1057D00084808583C9888187038470BD002C014043
:1057E00000340140828B22F008020A438283704712
:1057F00070B5028C22F480520284048C8288838BE0
:105800000D8823F4E6464FF6FF7303EA052535437A
:1058100024F400560C8903EA043434434E8803EA26
:1058200006362643094CA04202D0094CA04205D1BD
:1058300022F480448A8903EA82122243828085838B
:10584000C988A0F84010068470BD0000002C0140FB
:1058500000340140828B4FF6FF7322F4006203EAAA
:1058600001211143818370470185828270478288BC
:1058700022F07002828082880A4382807047A0F8FA
:105880004010704730B502881B4B1C4C98420DD01D
:10589000A0420BD0B0F1804F08D0194DA84205D0DE
:1058A000184DA84202D0184DA84203D122F070052D
:1058B0004A882A43154DA84206D0154DA84203D068
:1058C00022F44075CA882A4302808A8882850A8821
:1058D000028598420AD0A04208D00E4A904205D0D4
:1058E0000D4A904202D00D4A904201D1097A0186B8
:1058F0000121818230BD0000002C014000340140B4
:105900000004004000080040000C0040001000406F
:1059100000140040004001400044014000480140A4
:105920004FF6FF71818000210180C18041800172AA
:1059300070470029018802D041F0020101E021F006
:105940000201018070470029018802D041F0040162
:1059500001E021F00401018070470000234810B5E8
:1059600090F82010026801F01F00214951F8200032
:1059700020490242086802D040F4803001E020F45F
:1059800080300860C1031C484FF0000303D51B4959
:1059900091F8651039B31A4A01881488611A89B2DE
:1059A00001240F290BD3118801808168002900DAB6
:1059B0004942062903DD13490978022905D0417FB0
:1059C000012906D01188418010BD4477C377118822
:1059D000418041881288511A89B240F21A6291427C
:1059E000F2D3C47710BD437710BD0000F00500204E
:1059F00080930008B00200208C0C0020C40C002012
:105A0000340700202B0700202DE9F0414D680023CA
:105A10001E240F22854202DD0868BDE8F081D1F81E
:105A2000F450854202DAD1F8F000F6E701EBC20546
:105A30006D68854201DA134600E01446E218520808
:105A40005D1CAA42F2D101EBC20351F832505C68EE
:105A5000844202DAD3E9026701E053E90267001BDE
:105A6000C11789053A1B41EA9021D3178005FAF73F
:105A700059FB721BA0FB024601FB0261D31700FB1E
:105A80000310810241EA94502844C6E72DE9F04F03
:105A9000DFF8B8B16A48DFF8AC91DFF8ACA190F854
:105AA0000EC0BBF91A70BBF91C60BBF91850BBF9EA
:105AB0006C10BCF1070F48D2DFE80CF08D041A30EF
:105AC000485E7600D9F800208284DAF80020C2848B
:105AD000828CC38CA7EB820212B2A6EB83034A43EB
:105AE0001BB2594342F3CF2241F3CF23D11870E0C8
:105AF000D9F800204284DAF80020C284428CA5EB59
:105B0000820213B2C28C4B43A6EB820212B243F361
:105B1000CF24514341F3CF23E11814E0D9F80020FA
:105B2000C284DAF800204284C28C438CA6EB820245
:105B300012B2A5EB83031CB24A43614342F3CF2365
:105B400041F3CF24191949420AB244E0D9F80020A0
:105B50008284DAF800204284828C438CA7EB820294
:105B600012B2A5EB83034A431BB2594342F3CF223F
:105B700041F3CF24111914E0D9F800204284DAF857
:105B800000208284428C838CA5EB820212B2A7EBA8
:105B900083034A431BB242F3CF24594341F3CF223C
:105BA000A11849420BB216E0D9F80020C284DAF8F5
:105BB00000208284C28C838CA6EB820212B2A7EBF7
:105BC00083031CB24A4342F3CF23614341F3CF2204
:105BD000991849420CB2BBF91E50594605F21E569F
:105BE000A64201DACE8306E0A5F21E55A54201DDEC
:105BF000CD8300E0CC83B1F9204004F21E559542DC
:105C000001DA0D8406E0A4F21E54944201DD0C84F6
:105C100000E00A84B1F9222002F21E549C4202DA0A
:105C2000ABF8224008E0A2F21E529A4202DDABF825
:105C3000222001E0ABF82230417B8173BDE8F08F78
:105C4000B00200203C2401403C28014040050020D7
:105C50002DE9F04704467D487E4E002702787C48B7
:105C6000022AB0F9301004D0082A6ED0092A6DD06B
:105C7000E8E0C27B022A02D1B0F8402052B1A4F879
:105C8000421071810423B6F908101A460020FEF76D
:105C900003FFCEE07049DFF8C491DFF8C481496AA0
:105CA0000D14E5808068410216D5B4F9020040F277
:105CB000DA21884248DD40F26A41884205DD00BFB2
:105CC0000823B4F942101A4660E0A0F2DA20FAF78D
:105CD000A4FB0022634B68E0C0F3C001C0F30020C6
:105CE000DFF884A181420CD1D8F8440040F2BA41D7
:105CF00088426DDD40F66A118842E1DCA0F2BA40CC
:105D00004FE05A480078C0060CD5D8F8440041F25C
:105D1000243188425CDD41F2D4718842D0DC00F647
:105D2000DC4020E05248DFF84CA190F870100129C7
:105D30000DD090F86F00012809D099F80010C9071C
:105D400046D04D49098889B142E074E078E0B4F961
:105D5000020041F6DC6188423ADD42F234118842A9
:105D600010DC00F59270A0F500501AE0B9F91000AF
:105D7000B4F90210A0F59672914229DD00F59672F1
:105D800091420BDDB4F9421020231A460020FEF7A1
:105D900083FEA4F84200002817DB1BE0081A00F578
:105DA0009670FAF73AFB00225346FAF7A2FA0E224F
:105DB000FAF70EFBFAF768FB00B2C0F580406843C3
:105DC0008013A4F84200002D04DCA4F8427001E026
:105DD000A4F84250B4F842202848F280D8F8443061
:105DE0004364A0F84C20B0F93830254A3381D8F804
:105DF0005050B2F90420521B758B05EB620212B2AF
:105E0000F282002A00DCF78299F80020D20702D043
:105E1000B0F84E0006E0B0F94E20B6F91600824206
:105E200000DA1046708198F80A0008B1338109E061
:105E30005842308106E01348B0F87C00708100E0E1
:105E40007181378184F84070BDE8F0872B0700200E
:105E5000B002002064000020400500205809002006
:105E6000480100200000794000C092400C0700204B
:105E7000C40C002000C08240200000200409002043
:105E8000EA050020780A00202DE9F041B1F902501E
:105E900000232B241522854203DAB1F90000BDE866
:105EA000F081B1F9AE50854202DDB1F9AC00F6E700
:105EB00001EB8205B5F90250854201DD134600E091
:105EC0001446E21852085D1CAA42F1D101EB82058A
:105ED000B5F90230834206DA35F9026C35F9044C23
:105EE00031F9221006E01E4631F92240B5F906309C
:105EF000B5F90410801B091BC5178911AD0345EACC
:105F000090458703A1FB070CCA1702FB07C201FBE0
:105F100005219A1BD317FAF705F9000A40EA016038
:105F2000001900B2B0F5804FB9DB43F6FF70B6E759
:105F300070B5134C40F224452946204600F03EF847
:105F400000281BD0204600F0C7F82946204600F064
:105F50001DF80C4C00212046FBF706FB2046FBF702
:105F600081FBC0F164000849C0B20428087201D95D
:105F700000F046F9BDE87040FBF7BABB70BD000009
:105F800000380140580002407C0600200A0A012126
:105F90009140C943018070470029818902D041F4B2
:105FA000005101E021F4005181817047002A828A6A
:105FB00001D00A4300E08A438282704730B501F085
:105FC0001F0201240025C1F3421304FA02F2012B3F
:105FD0000FD0022B0FD0838A4FEA11210088134281
:105FE00004FA01F400EA040001D000B101252846BA
:105FF00030BD8389F0E7038AEEE710B5C1F34213A1
:1060000001F01F040121A140012B07D0022B07D072
:106010001430002A026805D00A4304E00C30F8E787
:106020001030F6E78A43026010BD000030B5044628
:10603000008A85B00D464CF6FF710840E98801439F
:106040002182A1894EF6F3100140A8882A891043C5
:106050006A890A431043A081A08A4FF6FF41084095
:10606000A9890143A1826846FDF758FF1948844277
:1060700001D1039800E00298A189090400EBC00156
:1060800001EB0010296801D5490000E08900B0FB50
:10609000F1F06422B0FBF2F109010B096FF0180571
:1060A0006B4300EB8300A3891D044FF0320306D538
:1060B00003EBC000B0FBF2F000F0070005E003EBDB
:1060C0000010B0FBF2F000F00F000843208105B093
:1060D00030BD0000003801408088C0F308007047E0
:1060E000F8B501210920FDF701FF01218803FDF723
:1060F000FDFE10258DF803502020ADF800001A4E4B
:1061000003248DF8024069463046FCF745F81649ED
:106110000C31086820F02000086018208DF803007A
:106120004020ADF800008DF8024069463046FCF78B
:1061300033F848208DF803008020ADF80000694650
:106140003046FCF729F88DF803502801ADF800001F
:106150008DF8024069463046FCF71EF80121042004
:10616000FCF76CF8F8BD0000000C014030B585B0BC
:10617000FFF7B6FF00244FF4E1300090ADF808407F
:106180000C201D4DADF80440ADF80A00ADF80640F6
:10619000ADF80C4069462846FFF748FF25208DF8EA
:1061A000100004208DF811008DF8124001208DF8A8
:1061B000130004A8FDF77EFB012240F2244128468B
:1061C000FFF71BFF01212846FFF7E6FEFBF7BAFAAF
:1061D000012280212846FFF7E9FE012240212846BE
:1061E000FFF7E4FE012202210448FBF74FFAFBF718
:1061F000A9FA05B030BD000000380140440002405B
:1062000070B51D4D00242878432834D1687846287D
:1062100031D1A878502807D0512805D0812803D043
:10622000892801D0212826D1144E7071E978717225
:10623000A81C891CFAF7B8FEB072717A2944097952
:106240003182884217D106F10E00017841F0020137
:1062500001700B48016841F020010160317A094862
:10626000002204E02B5D03552A55641CE4B28C42E5
:10627000F8D38078707170BDC40700207C060020C0
:106280000C0C0140F60B002070B51D20FDF7F1FA53
:10629000FDF774F91D20FDF702FB154890F82F104B
:1062A000144D0623144C85F8381090F83B1095F8DF
:1062B0003B201143012A04D0022A07D0042A0AD025
:1062C00010E0827A8A420DD0007B09E0027D8A428A
:1062D00008D0807D04E0827F8A4203D090F82000BD
:1062E000884200D12370002085F8400070BD000076
:1062F00060040020480100202B0700200B480021EB
:106300004180A0F1B8018A898280CB891A44C28079
:106310000B8A1A4402814B8A1A444281898A1144A9
:10632000818143F6FF71C1817047000000020020A7
:10633000084940F61C72B1F90C00904202DA00F5EF
:106340009F7005E041F2E302904201DDA0F59F70ED
:10635000C88170476400002038B51348C16941F016
:106360000401C1611E208DF8000002208DF801009B
:106370008DF8020001248DF803406846FDF79AFA73
:106380000A4984200880094947F690602C3108802A
:106390000020091F0880054914310C80091F08805E
:1063A000081F048038BD00000010024000080040B3
:1063B00030B420491E4A45788B7A114692F83B400A
:1063C00091F83910AC4218D14BB10379994202D0FF
:1063D0004379994201D140791AE0807909E08379C3
:1063E000994202D0C479A14202D182F82F3011E043
:1063F000407982F82F0030BC7047C578AC42FAD1A2
:106400006BB1C379994202D0037A994205D1007ADF
:1064100082F82F0030BCFEF7E1BB407AE9E7437A0F
:106420009942E2D00479A142DFD0007AE1E700008E
:106430006004002048010020FEE700002DE9F0473D
:106440000446007F012868D13548E1880288511A46
:1064500089B2072916D30088E080B4F9000044F21D
:10646000DD414843401346F6D96148438013A0609C
:10647000401000B2A0814FF08051B1FBF0F0F9F76D
:10648000C7FF2061B4F90C6096B1B4F902104DF663
:10649000B05048430014A082B4F904704DF6B052D5
:1064A00007FB02F24FEA2245E58204D4024603E0EC
:1064B0000020E08330E0424212B22283002D01DB53
:1064C0002B4600E06B421BB2DFF85890638398467E
:1064D0004FF4804AB24208DAF9F791FF2169F9F7DF
:1064E00064FEF9F7B8FF801304E0002901DA48469A
:1064F00000E05046E083B04509DA2846F9F77FFF0F
:106500002169F9F752FEF9F7A6FF801304E0002F86
:1065100001DA484600E050462084BDE8F0870000DC
:106520003407002000C0FFFF70B531480022324C14
:1065300001783048022905D1C17B022902D1B0F887
:10654000401021B1008EA4F84E00228770BD90F853
:106550000D31284890F846102748B0F8440000B2A2
:106560007BB1264B43F6CC45B3F90430AB4228DB74
:10657000022918D0224900BFFBF766FCA4F84000AE
:1065800021E00229F6D11F490978C1F381010129CF
:1065900004D0022904D01A496C39EDE71A49EBE717
:1065A00019496C31E8E716496C39FBF74DFC80B2AC
:1065B00040F2D271A4F84000884204D3A4F84010FD
:1065C00001E0A4F840200C49B4F8400048313834C8
:1065D00001F086FAB4F91400B4F912204142514393
:1065E00089132180B4F9101048438013E08270BDF4
:1065F0002B070020B002002004090020EA0500203B
:10660000D08D0008D80400208C8C0008034800219D
:1066100080F82A10C1830187704700000409002018
:1066200010B504000B462D4AC3F1000028D5644282
:10663000002B12DAA04207DA214600F02DFA32F8D8
:106640001000C0F5404041E00146204600F024FA29
:1066500032F8100000F5004038E0A34208DA214685
:10666000184600F019FA32F8100000F540402DE00D
:10667000204600F011FA32F81000C0F5803025E015
:10668000002B12DAA04207DA214600F005FA32F8B0
:10669000100000F5804019E00146204600F0FCF9AA
:1066A00032F81000C0F5004010E0A34208DA21469D
:1066B000184600F0F1F932F81000C0F5804005E00E
:1066C00053B1204600F0E8F932F81000B0F5004F61
:1066D00001DDA0F5803010BD002010BD488F0008FE
:1066E00040438013494300EBA13000220302002BFA
:1066F00014DDB3F5001F01DC802001E04FF40050F1
:1067000093FBF0F1014401EBD1714910814206D0B5
:10671000521CD2B20846062AF2D300E00021C8007B
:1067200000B2704702E008C8121F08C1002AFAD15F
:1067300070477047002001E001C1121F002AFBD101
:10674000704700002DE9F047A74CA848218802882F
:10675000511A89B20F297DD30088A4F13C0520800D
:10676000288F08B1401E288795F800C0A04ACCF3B6
:10677000810001281DD0022820D0D18B9D4E9A483F
:10678000DFF87492F388407E0027B1F5926F1CD831
:10679000142818D37820607643F01000F08040F27F
:1067A0006660A8812CF001002870D77389F800700A
:1067B00018E0D08B00EB4000C00302E0D08B8F4983
:1067C0004843010CDAE7401C04E0B1F5DB6F09D364
:1067D00010B1401E607605E023F01000F0804CF010
:1067E00001002870B5F90200B5F914304143C3EB3C
:1067F000C303C1F38F31C3F3D10303EB510109B2DA
:10680000A9829046D28B4FF080535043B5F91620A1
:10681000C0F38F30C2EBC202C2F3D10202EB5000D0
:1068200000B2E882AA6A42431213EA6293FBF2F2D0
:106830002A63734A1080A2680A44A260E168014496
:10684000E160207C401CC0B22074072802D942F3CA
:10685000CF0000E0C5E02883C9106983E760A76026
:1068600041F6C8012774884204DD298B654AB2FBD2
:10687000F1F1E981C117890341EA9041800342F6B1
:106880009B420023F9F74EFCA88457485E49A0F1CB
:106890003C002A78B0F906005FEA827C00FB01F137
:1068A0004FEA2143C2F3810115D5012907D00229FE
:1068B0000BD04FF2685141430914A18011E049F611
:1068C0008C4148430014A08020E04CF6183141432D
:1068D0000914A18026E001290ED0022918D0A08039
:1068E0006B844A4948430014A4F81E00FBF7CCF817
:1068F00047480088C0B143E04AF65C31414309147F
:10690000A1804BF62C21484300146884E383EDE713
:106910004DF2AC5141430914A1804EF27C414143F8
:10692000091469843B49DDE795F8200000BB88F82D
:106930000F7089F80070B5F91A00A0F50C519F3955
:10694000B1F56E7F18D8617FF42912D93249E880F9
:106950002E4AA1F8460050430014A880A1F8440034
:10696000FF2085F8200081F828002C493C20087081
:1069700006E0491C617703E0607F08B1401E607744
:10698000B5F91A10B4F91E0081420EDDA07E7D28F3
:1069900009D9F08840F00800F0802148017821F002
:1069A000020101700EE0401C06E0A0F23D108142A1
:1069B00008DAA07E10B1401EA07603E0F08820F037
:1069C0000800F080B5F91810606908446061217E04
:1069D000491CC9B221761F2903D94011A8836761D8
:1069E0002776BDE8F087000014050020340700205A
:1069F000B0020020640A00202B0700203033010081
:106A0000180A002074E8260BCC0E0100488501000E
:106A100036070020D0450100C40C002028070020C4
:106A2000EA050020024941F68B3088627047000079
:106A3000D804002070B5164C06252078062825D2EB
:106A4000DFE800F003080E141A211248FAF7EAFAF8
:106A5000012016E00F48801DFAF7E4FA022010E04A
:106A60000C480C30FAF7DEFA03200AE0094812302D
:106A7000FAF7D8FA042004E006481830FAF7D2FAF8
:106A80000520207070BDFAF7EDFA2570257070BDF5
:106A90002C0700203C8E0008090A05D0B0FBF1F05D
:106AA000FF2800D9FF20704700207047D0E900215F
:106AB000C368521A5A4301EBA231816041607047AA
:106AC000B0F90020B0F90210B0F90630521A5A435A
:106AD00001EBA231818041807047000030B5494B05
:106AE000188849490A8A801A85B24848484A0F2DB1
:106AF000047801F150001DD31D880D82117A090719
:106B000013D5022C01D0434912E0434DB0F90210D5
:106B1000B5F90050A94205DC02DA01F1020108E0F2
:106B2000458007E0A1F1020103E0022C02D13B49BC
:106B300009884180B0F840101D88691A89B29C29E3
:106B400049D31988A0F84010916A0023B1F5804F0D
:106B500031DB3349096DB1F5405F2CDD314940F23D
:106B60006665B1F91010A94212DD43F69915A942E4
:106B700002DB40F2333108E040F23335A1F26661C6
:106B8000694343F2333591FBF5F1A0F8441001E07D
:106B9000A0F844302449B2F806510978C1F38101C4
:106BA0002DB100BFB0F8441001F21E511CE092F864
:106BB0004620022A10D0A0F84430022C01D0A0F8C0
:106BC0004430B0F95C10B0F9443001F114029A423B
:106BD0000DDAA0F85C2030BD012901D00229E1D1F5
:106BE000B0F8441001F23331A0F84410E5E703F1A6
:106BF0001402914203DD1439A0F85C1030BDA0F8F6
:106C00005C3030BD34070020140000202B0700202A
:106C1000B0020020D6040020D4040020D0040020BC
:106C20004801002040050020D80400202DE9FC4147
:106C300001210220FDF742F901211920FDF756F943
:106C400001213C48FBF7FAFA4027ADF80070032415
:106C50008DF802400420384D8DF80300694628461F
:106C6000FBF79AFAE001ADF800008DF802401C2015
:106C70008DF8030069462846FBF78EFA4FF4E07161
:106C80002846FBF710FBA815ADF800008DF8024070
:106C900010208DF8030069462848FBF77DFA4FF471
:106CA000A060FCF739FE1D208DF8040001268DF848
:106CB000056000258DF806508DF8076001A8FCF7E7
:106CC000F9FD1F498C2008801D494FF6FA702C31C0
:106CD00008806E20091F0880194814300680184863
:106CE00008300780164920310D80154AD020121D2A
:106CF0001080134A45F2F300183210800A1F45F243
:106D0000500010800E4A4FF6FF7038321080121D6E
:106D10001080121D108041F21B10088000F012F844
:106D2000FBF73EFD064810300580001F0480BDE8DB
:106D3000FC810000000C1A0000100140000C014012
:106D40000004004070B51D20FCF788FD2A4D40214D
:106D50002846FBF79FFA840080212846FBF79AFA21
:106D600044EA4004A9152846FBF794FA0443E0B22C
:106D7000224C84F83C00FBF719FB0546052805D991
:106D80001F48C18841F04001C18001E084F83850BB
:106D90001C48007A000703D594F838001A490D5CA6
:106DA0004FF6FA702063E062A06260622062E061E8
:106DB000A0611648606300206064206584F83F008D
:106DC00084F84000FBF7A0FAA07AFF2811D0022037
:106DD00084F83D000E480088A0662846FBF742FF75
:106DE000207820F001002070BDE870401D20FCF7E5
:106DF0004BBD0120ECE700000010014048010020DD
:106E0000640A0020B002002044980008DCFF05005E
:106E1000240400402DE9F0434E484F4902880B8876
:106E20009A1A92B20F2A69D3098801804B49098BBB
:106E3000027D00EB42029180017D491CC9B20175BF
:106E400008295BD3002404752246017D00EB410331
:106E5000491CB3F90430C9B202EB630212B20175E6
:106E60000829F2D33E4904753E4B4A8044800E788F
:106E70009D895FEAC67C40F638694FF0030714D05D
:106E8000A2F22B5C42F6E858C44520D3A1F1020CD3
:106E900026F00204ACF8002047750C7040F22B5429
:106EA000A24211DA45F004021EE046F001060E701F
:106EB0004A4507DD45F001029A8126F002020A7078
:106EC000477519E0447517E045F002020CE04A45A9
:106ED0000CDA8775427D12B1521E42750CE046F005
:106EE00002020A7025F007029A8105E0B30703D574
:106EF000837D2BB15B1E837540888880BDE8F0835D
:106F000042F6AA239A4222DAB1F904302BB941F2AF
:106F1000CD05AA4201DA4480EEE7134C920302EB5E
:106F2000843241F67244B2FBF4F214B24FF480554D
:106F300002464480AC4200DA5580B2F90240E41ABD
:106F400004F5A374B4F5237FD6D84380D4E74FF477
:106F50008043FAE7F80A002034070020B00200203E
:106F6000EA050020640A0020C8F1FFFF2DE9F04186
:106F70006D4CDFF8B8E14FF0000594F83410C80705
:106F800006D094F938104B42002958DD0E4657E0E0
:106F9000674884F83750A4F84250664A90F83800A1
:106FA00084F840001586CEF80450CEF80850624EA2
:106FB00040F26663CEF80C50A4F87C3036F810002E
:106FC0005E4E768830444FF6FF7606EA800024F85D
:106FD000300B4FF0806044F8040CA32020846084C0
:106FE0005810A084E38440F69910208558006085ED
:106FF0004FF48050A08541F23330E08541F2666065
:10700000208641F69910608641F6CC40A0864FF468
:107010000050E08642F23330208742F2666060879B
:1070200042F69910A08742F6CC40E08782F89D5046
:1070300041F00100207184F84450BDE8F0811E4603
:1070400094F937004242002801DD074600E0174668
:10705000F61B012E0BD0002800DB02465FFA82F6F9
:1070600084F8380094F84F00012805D041E0002949
:1070700000DA1946CEB2F3E794F939305942002BC1
:1070800001DB184600E0084694F93A20C7B25042A6
:10709000002A01DB944600E08446BC4508DD002A56
:1070A00000DA0246D7B2002B00DA0B46D8B207E06E
:1070B000002B00DA0B46DFB2002A00DB1046C0B21C
:1070C00004EB4000B0F9501004EB470030F9502FAA
:1070D00011444910018084F84F5084F83E5084F8E0
:1070E0003D5084F83C5084F83B5084F83A5084F882
:1070F000395004EB46007546B0F9500024F8420FB1
:10710000BEF80410C82309B26422FDF7C5FC68600C
:10711000E968401AA9680844A860B5F90010484316
:10712000C013E860608788E7780A0020D80500204F
:1071300048010020B002002056980008640000209A
:10714000F0B4544890F83410C90776D0524990F8FA
:107150004030002291F838108B426FD04F4CA0F88D
:1071600072204F4DE65C04468E4294F9374002D0BF
:10717000EE5C8E420FD1641C64B280F83740EB5C49
:107180008B4202D1641C80F8374090F937300F2BC6
:107190001BDD0F2317E0434DEE5C434D8E4202D0C2
:1071A000EE5C8E4211D1641E64B280F83740EB5C15
:1071B0008B4202D1641E80F8374090F937406FF05F
:1071C0000E039C4201DA80F83730324B90F83F5082
:1071D000393390F83740EC5490F83F305B1CDBB209
:1071E00080F83F30062B01D380F83F2090F93940DA
:1071F00090F93B309C420ED190F93D40A3420AD118
:1072000090F93A4090F93C309C4204D190F93E40CC
:10721000A34200D1012280F84F201F4A80F840107D
:1072200090F937501378214A012D0DDD14465E0781
:10723000A46804D544F0080403E028E015E024F035
:107240000804946080F83510B5F1FF3F0ADA5B0757
:10725000936802D523F0080301E043F0080393602C
:1072600080F83510F0BCFBF74FB890F84F100129AB
:107270000DD1B0F8721043F60953491C89B2A0F839
:107280007210994203D9A0F8722080F84F20F0BC08
:1072900070470000780A0020480100203898000854
:1072A0003E9800084A98000850980008B002002054
:1072B00010B5D0E900210369114481FB03318C0230
:1072C00044EA93514260D0E9022382FB03329402E4
:1072D00044EA93521144816010BD000030B520494A
:1072E000204AB1F86A301088C01A80B20F2836D30D
:1072F0001088A1F86A001C4D00204FF000432A5C62
:10730000940903D00124B4EB921F24D1D20622D0D9
:10731000164A52F820201268134C123434F81040E8
:10732000224201EB000494F9722008D00A2A04DBFF
:107330000A6823FA00F4224308E0521C09E012F123
:107340000A0F05DC0A6823FA00F4A2430A6002E08F
:10735000521E84F87220401CC0B21128CFD330BD19
:10736000F0050020340700204C9300084C940008DE
:107370002DE9F00779497A480A8903889A1A92B266
:10738000082A74D300880881A1F12C0042890AB12F
:10739000521E4281734A92F82820802A67D302F055
:1073A0003F020A70C2890AB1521EC281B1F9062099
:1073B000902A0CDB8A46FF2A09D08146C089002822
:1073C00055D1694800230078092805D005E0BDE8BB
:1073D000F007624800F09AB90823644A92F8EA502C
:1073E0000DB143F004036248817AC90701D043F02C
:1073F0000203D2F808C05FEA0C5101D543F0010343
:10740000176800215B4EFC0302D596F8654004B175
:107410008021C4885FEA446801D541F040015FEAF9
:10742000845801D541F020015FEAC47801D041F0D1
:107430001001007A400701D541F008014E4800785C
:10744000C00701D041F00401A00601D541F00101BF
:107450000020012D00D1082096F8705085B992F8CF
:107460004620022A04D0012A05D03AB108E072E091
:1074700040F0030004E040F0020001E040F00100B1
:107480007A0701D440F02000CCF3C0020025CCF3F1
:10749000002C624502D13A0700D4042596F86F20EB
:1074A000012A01D145F00105344A0027BC46127873
:1074B0003E46C2F38102012A04D0022A04D0032AE4
:1074C00004D004E0022602E0042600E010262C4A44
:1074D00064060ED5214C1C342478240609D5147872
:1074E000640606D4274A40F6CC44926D6243140CDD
:1074F00005E0B2F8B62040F699146243940B4FF0C1
:1075000008088AF80A804FF061088AF80B808AF828
:107510000C308AF80D108AF80E008AF80F508AF89D
:107520001070270A4B4083F06901414069408AF896
:10753000117079408AF81240614052468AF813C0AF
:1075400071408AF8146051754FF4C871A9F80E1093
:10755000FF20AAF80600BDE8F0077047F0060020FB
:1075600034070020F00500202B070020B002002087
:10757000640A0020C40C002058090020D804002010
:1075800048010020280800205048816941F0FC0192
:1075900081614FF4A060FCF7BFF9FBF78FF9FCF7AE
:1075A0001FFBF9F7FDFAFCF715F9FDF77BF9FFF77B
:1075B0003DFBFCF755F8FFF7C5FBFBF7F1F8444D31
:1075C0004FF40050A5F81601FEF7D0FD00214FF44E
:1075D000FA5340F2EE220020401C80B29842FBD3C6
:1075E000491C89B29142F6D33A48002680F872606D
:1075F000F9F76CF9F9F708FEFCF722FBF9F7E0FC64
:10760000FEF7AAFE102234493448F8F7BCFD01F019
:10761000DDF9334C344FE08820F04000E080314801
:10762000017821F020010170FA20F8814FF4967062
:10763000E887FFF7F7F92D492D48FCF77EFA2D482A
:10764000FCF7A0FA2C48416A88472C48416B8847D0
:10765000FEF7DCFF2A48FAF713FA2A494220C880CD
:107660002949C8603E71E088E081208920826089D4
:107670006082FAF709FDFAF76BFCFFF763F801F097
:1076800045F9FFF7C7FB00F0F9F9FFF727FE01F016
:1076900001F8FEF763F9FAF7C7FAFBF701FBFFF70A
:1076A0001DFAFCF709FDFAF723FFFAF755FF00F082
:1076B0007BF8FFF75DFE1248FAF78EF800F06AFAE1
:1076C000FDF734F9FAF712FACDE700000010024096
:1076D000B002002040050020C40C0020300600202D
:1076E000640A00204801002028070020D408002058
:1076F000A40800201404002038000020E40000202A
:10770000E40900205407002048040020F0B5234974
:107710000278B0F9064000231F4E31F81210FF2CFA
:1077200018D0B0F904701E4DBC4231DA00EBE4070A
:1077300004F00704BF7AA7408478FFB23CB190F808
:1077400001C0ACF1010C64451FDA3C061DD455F8AC
:1077500022200DE056F82220116012498A79521C2D
:10776000D2B28A71022A02D38370C3808B71F0BDBA
:1077700011608178491CC9B2817042789142F6D378
:107780008370C188491CC180F0BD56F82220EFE704
:1077900055F822201160F4E72C9500085E9300084C
:1077A000D4940008C4060020F0B561486149B0F8DF
:1077B0006C200B889A1A92B29C2A7BD30988A0F875
:1077C0006C105D495D4F91F82A1001F0070297F89F
:1077D0004610022A00D1491E594C80F83E104FF045
:1077E0000203E2884FF00001550401D5012236E082
:1077F000A489E50601D5062231E0250701D5082236
:107800002DE0550603D44F4D2D78AD0601D5042249
:1078100025E0150501D5072221E0150601D50A222C
:107820001DE0950601D50C2219E0150701D50B22A4
:1078300015E0550701D4D50501D510220FE0D50676
:1078400001D505220BE0650703D4A50701D4E407A1
:1078500002D080F86E3007E0920403D5032280F84E
:107860006E2001E080F86E10374A384C92F820E024
:10787000324A251FD2F808C02D4AB2F87060721C37
:1078800092B2BEF1000F0DD02CF4000CC7F808C066
:1078900090F86E70B7B11E2F1AD090F86F200AB30F
:1078A00025E007E04CF40006BE60A0F870200A2A2C
:1078B00001D22360F0BD142A01D22B60F0BDA0F8E4
:1078C0007010F0BD2B60A0F8701080F86F10F0BD44
:1078D000642E04D2A0F87020322AEED3E9E7A0F893
:1078E0007010EAE77F1C80F86F70A0F8701090F8B5
:1078F0006F20012A10D0002AE9D0B0F87060761C01
:10790000B6B2A0F870601E2ED7D323603C2EDED90D
:10791000521E80F86F20D2E7B0F87020521C92B24D
:10792000A0F870202360C82AD1D980F86F10C6E76C
:10793000F005002034070020C40C0020B002002015
:10794000640A002048010020D8040020141C0140D3
:10795000F0B54248B0F84810491C89B2A0F8481068
:1079600002297AD33E490024A0F848400A783D4BCA
:10797000042A57D04FF48041082A0BD0A0F10C0202
:10798000B2F900208A4200DA1146B3F980208A4217
:1079900000DA1146344A92698A4200DA11B2418211
:1079A00082881D8AC2EB8502304D12B22D78C5F354
:1079B00081062A4D42F291767243B5F976509212C1
:1079C0006A431213C26086681546C6EBC60642F3C8
:1079D000D102F60202EBA6328260C66C1644C6647F
:1079E000B0F850707F1CBFB2A0F85070B7F5806F30
:1079F00004D3B6120682A0F85040C464891A1C4E03
:107A0000C26A724340F255564E4302EB4602466A42
:107A100032444262B3F93030B2EB034F06DD1A0450
:107A2000426206E01349B1F90410B3E7002A00DA14
:107A30004462C162104990F83D2091F838108A42A2
:107A40000BD080F83D10B0F84210A0F84410B0F808
:107A50004010A0F84210A0F84050F0BD40050020B2
:107A60002B070020B00200205C0C0020D80400206E
:107A7000C3F5FFFF780C0020480100201548164987
:107A8000B0F85A200B889A1A92B20F2A20D309888C
:107A9000A0F85A10B0F9001041F630225143891372
:107AA000A0F86C100D494FF480420B78A0F10C0146
:107AB000022B06D1B1F90030934202DA1B1D0B8074
:107AC00000E00A800021A0F8601020F85C1F4280CE
:107AD0007047000040050020340700202B070020DD
:107AE0004FF6FF7202EA800210F4404315480ED0B0
:107AF000B3F5804F14D0B3F5004F4FEA122216D0E1
:107B0000C2F5807330F813305B424B8005E0120AF7
:107B100030F812304B80C2F5807230F812000FE05E
:107B2000120AC2F5807330F813304B8005E030F84C
:107B30001230C2F580725B424B8030F81200404236
:107B40000880704748910008104A518A908AD28A6A
:107B500016384639A2F1110200D54942002A00DA4E
:107B600052421144002800DA40420844084943F6D2
:107B7000284300B2B1F936205A43921340F2D7336A
:107B8000584302EBA030C88670470000B0020020C6
:107B900040050020F0B5904990480A8903889A1A58
:107BA00092B23E2A1ED30088088101F138004FF4BA
:107BB000FA63428A9A4202D2521C428200E0438215
:107BC000874A92F82220802A0CD302F03F020A70E2
:107BD000B1F90620402A06DBFF2A04D0C2883AB158
:107BE000521EC280F0BDBDE8F0407B48FFF78EBD5D
:107BF000428A9A42F6D307784FF0010E3A074FF0C7
:107C0000FF055BD5847A40F2DC52630708D444F068
:107C100004038372C28081F80BE081F80AE04CE033
:107C20004378072B05D0032B03D0052B01D0062B5F
:107C300007D1660605D444F040038372C280052252
:107C400039E0654A5FEA437C02F138024FF420765E
:107C5000127A0DD55FEAC26C0AD45FEA446C07D48D
:107C600042F0100202723A0628D4C680192222E09D
:107C7000DF0709D0970707D4670605D442F0020250
:107C80000272C680042216E09F0709D5170707D4A1
:107C9000670605D442F008020272C68003220AE099
:107CA0001B070BD5530709D4630607D442F004021F
:107CB0000272C6800B22CA728A72CD80494AB2F91A
:107CC0002230B2F91A7003F23D140022A74200DB01
:107CD0000276414E444C06F13806A479B6895FEA33
:107CE000C46C06F101064FF4C874B6B213D5868190
:107CF000B6F57A7F05D9017A21F08001017282817F
:107D0000F0BD037A1E06FBD4828143F0800202722A
:107D1000C480112035E09F4216DA037E052B13D272
:107D20008681B6F5487F04D98281027A22F040022A
:107D30000272027A5606E3D45B1C037642F04002DC
:107D40000272C48002201CE0284B1C89C4F3C006C8
:107D5000C4F3002740F2EE24BE4216D11E78360747
:107D600013D4427E012ACBD1428BB2F5167F02D2C8
:107D7000521C4283F0BD827A42F002028272C480B9
:107D80000F20C8728872CD80F0BD93F80D714FF44A
:107D90000046012F18D1164F41F6583C7F6C6745BD
:107DA00012DD83F80CE1134B1E60C38AA34202D29A
:107DB0005B1CC382F0BD4FF4FA73C3801C23CB72EB
:107DC0008B72CD80C282F0BDC2820A4883F80C213A
:107DD000001F0660F0BD0000D4060020340700201C
:107DE000F0050020D8040020640A0020B002002022
:107DF00048010020140801402DE9F05FFD48FE49CC
:107E0000DFF8F8A3007E0A1D131D012850465ED03E
:107E100030F85A4F0C8041881180BAF85E00188003
:107E2000FDF734FEF64DF74C49F2CD32B5F91E1090
:107E3000A183B5F9200043F6CC4C01EB4000504340
:107E40000014E083B4F92230B4F9206000FB03F29F
:107E500001FB062242F38F326282B4F9187070433C
:107E600007FB0CF740F2333CBF1302FB0CF207EBAD
:107E7000A23201FB1300228340F38F30A082B4F9B9
:107E80001A1043F6AE72514300EB0012891302EB55
:107E90008010DD4F01EBA030DC4E6083786C3060E9
:107EA000316930468847DA49308948800846FDF70D
:107EB000CFFEDFF860B301264FF000099BF8000009
:107EC00008280CD0618F218204284AD01AE030F8AB
:107ED000604F0C8041881180BAF864009FE7CE485B
:107EE00090F93710491C022939D890F8741019B14B
:107EF000B4F85A00208205E0618F2182A4F85A105C
:107F000080F87460B4F91410B4F90A00C34AF9F7A0
:107F1000B5FAE062BAF91611884204DDBF48E162A1
:107F2000027C91408162B748DFF8F4E2503847F2B2
:107F3000A30802784EF24611002A7AD0012A79D09D
:107F400080F800909BF8000004280DD0B34AB4F9E3
:107F50001210B4F90800303AF9F790FA08E0608F8F
:107F6000C8E7686A0014E062B87A002863D0AD48B8
:107F7000A3462546A062A94C443C2060E86A6060A4
:107F800020461035FCF772F89E4928883C39FFF7E7
:107F9000A7FDDFF87082A8F15008D8F81410C8F8CF
:107FA0007010B5F91010A068B5F9123000FB01F798
:107FB000E268584302FB137444F38F3702FB01005D
:107FC000AF8740F38F34EC87974D28466F80AC80A5
:107FD000FEF734FA287F08F11805012871D06042B5
:107FE00041104DF6B350474369803A142A80404609
:107FF000A8F804408B18C380891AA8F808108AF8DA
:108000000C90B8F904305446002B00DD2673B8F903
:108010000600002802DD217B891C2173B8F90820A5
:10802000002A02DD217B091D2173217B072979D2DA
:1080300002E007E02CE05AE0DFE801F07470886E9F
:1080400084728600B5F91E2042448A420AD8B5F9E6
:10805000202042448A4205D8B5F9222042448A426F
:108060007FF670AFA0F80290B7F8B6204946B2F597
:10807000C87F01D8467006E0B2F5487F01D80222D9
:1080800000E0032242708AF80F108BF8001025E000
:1080900080F80090B5F91EC04A46C4448C4509D802
:1080A000B5F920C0C4448C4504D8B5F922504544E4
:1080B0008D42D5D9B7F8B610B1F5C87F02D8467051
:1080C00007E017E0B1F5487F01D8022100E0032165
:1080D000417042808AF80F208BF80020BEF806100D
:1080E00041F40061AEF80610F9F724FF2AE74FF4D7
:1080F000AF703DE74C484DF6B352B0F920305942CD
:1081000049106980B0F91E00504302142A8040468D
:10811000A8F804306EE705E0667303E0022100E092
:10812000032161739BF80010404E0129404F617B91
:10813000DA460DD007297DD2DFE801F07CFDFCFB9B
:10814000FAF9F8000421ECE70521EAE70621E8E75F
:108150000729F0D2DFE801F06E0429799ECCF800FF
:1081600001461846FBF7D0FC2860B5F9020040F63E
:108170008151484380136880B5F9001040F6815260
:108180005143891329804218A2F68152B8F80E3063
:108190005242C3EB620212B2A8F80C20002A01DCA2
:1081A000A8F80C90B8F80C2067E1404201B25042A8
:1081B00000B2FBF7A9FC2860B5F9020040F6815136
:1081C000484380136880B5F9001040F6815251434E
:1081D000891329804218A2F68152B8F80E30524213
:1081E000C3EB620212B2A8F80C20002A01DCA8F846
:1081F0000C9020E0E4090020342C0140B002002063
:1082000040050020640000204801002048040020B0
:10821000040400202B070020780A0020D408002046
:10822000640A0020A2FEFFFF180A0020002401407B
:1082300000280140C6E0B8F80C204CE13046F8F7C1
:108240000DFD01231A460721B1E019461046FBF740
:108250005BFC2860B5F9020040F681514843801369
:108260006880B5F9001040F6815251438913298086
:108270004218A2F68152B8F80E305242C3EB6202A5
:1082800012B2A8F80C20002A01DCA8F80C90B8F86B
:108290000C204DE15942404209B200B2FBF734FCD8
:1082A0002860B5F9020040F6815148438013688088
:1082B000B5F9001040F681525143891329804218C4
:1082C000A2F68152B8F80E305242C3EB620212B2EB
:1082D000A8F80C20002A01DCA8F80C90B8F80C20B3
:1082E00056E13046F8F7BAFC01231A4605215EE054
:1082F0001146FBF709FC2860B5F9020040F68151F0
:10830000484380136880B5F9001040F6815251430C
:10831000891329804218A2F68152B8F80E305242D1
:10832000C3EB620212B2A8F80C2006E06FE143E151
:1083300014E1E5E0B5E088E006E0002A01DCA8F8F9
:108340000C90B8F80C204EE1504201B2584200B2F5
:10835000FBF7DAFB2860B5F9020040F6815148438B
:1083600081136980B5F9000040F6815250438013B3
:1083700028800A18A2F68152B8F80E305242C3EB98
:10838000620212B2A8F80C20002A01DCA8F80C90B6
:10839000B8F80C20A4F85C201144A4F85E1008443E
:1083A00055E13046F8F75AFC01231A4606213846B3
:1083B000F8F754FC01213046F8F7C6FB0121384696
:1083C000F8F7C2FBB04EBAF8080055463080BAF84C
:1083D0000A007080BAF81000B0803046F9F75EFAF3
:1083E000B4F85A00F1880844A4F86000B4F85C00BE
:1083F00031890844A4F86200B4F85E007189084429
:10840000A4F86400317EA148012978D034F85A1FBD
:10841000018061884180A18881809C49028808315F
:108420000A8042884A80808888809848896A083013
:10843000884795F83E0000287ED0F8F713FE15F81F
:108440003E0F401E2870BDE8F09F01461846FBF71E
:108450005BFB2860B5F9020040F681514843801368
:108460006880B5F9001040F68152514389134218D3
:10847000A2F68152524229805208A4F85E2010448C
:10848000A4F85C000844A4F85A0000213046F8F72C
:108490005BFB00213846F8F757FB01231A460621FB
:1084A000CCE6404201B2504200B2FBF72DFB2860FF
:1084B000B5F9020040F68151484380136880B5F950
:1084C000001040F68152514389134218A2F681529E
:1084D000524229805208A4F85E201044A4F85A00A1
:1084E0000844A4F85C0000213046F8F72DFB002179
:1084F0003846F8F729FB01231A4605219EE6B4E029
:1085000019461046FBF700FB2860B5F9020040F65B
:108510008151484380136880B5F9001040F68152BC
:10852000514389134218A2F68152524229805208BF
:10853000A4F85A20104400E09AE0A4F85E00084431
:10854000A4F85C0000213046F8F7FEFA0021384616
:10855000F8F7FAFA01231A460721C2E659424042C7
:1085600009B200B2FBF7D0FA2860B5F9020040F674
:108570008151484380136880B5F9001040F681525C
:10858000514389134218A2F681525242298052085F
:10859000A4F85A201044A4F85C000844A4F85E0033
:1085A00000213046F8F7D0FA00213846F8F7CCFA27
:1085B00001231A46062194E61146FBF7A5FA286026
:1085C000B5F9020040F68151484380136880B5F93F
:1085D000001040F68152514389134218A2F681528D
:1085E000524229805208A4F85C201044A4F85A0092
:1085F0000844A4F85E0000213046F8F7A5FA0021EF
:108600003846F8F7A1FA01231A460521C9E6504277
:1086100001B2584200B2FBF777FA2860B5F90200C0
:1086200040F68151484380136880B5F9001040F648
:108630008152514389134218A2F681525242520884
:108640002980A4F85C201044A4F85E000844A4F833
:108650005A0000213046F8F777FA00213846F8F73B
:1086600073FA01231A4607219BE634F8601FCFE610
:1086700007480088A0F5D04168393FF4E4AEBDE872
:10868000F05FF9F7A5BB0000E409002030000020EE
:10869000182C01402DE9F041904C9148B4F862103B
:1086A0000288511A89B20F296FD30088A4F862009A
:1086B0008C480088DFF83082C0074FF000054FF08B
:1086C000010741D0874AD4E90C1024321388B1EB5A
:1086D000530F02D21288511A08444FF4F3718842A2
:1086E00000D208468149B1FBF0F0616CC1F3510141
:1086F000084406466064F7F790FE00227C4BF7F7CB
:10870000F8FD4FF040427B4BF7F7F3FD0E22F7F7F1
:108710005FFEF7F7B9FEA4F8AC0094F86D00401CBA
:10872000C0B284F86D00082834D36C4898F846200D
:10873000001F03789A4201D0027045806E4A137878
:108740006E4A23B1458021E06564256558E0D8F87C
:108750009410A1F5FA618E4211DDE16D8B1C9E42F1
:1087600005DDB0F902100A290DDA491C06E08E4237
:1087700005DAB0F90210002908DD491E4180B0F980
:1087800002000A2802DB177001E0A2E01570E6651E
:1087900084F86D505A484FF4A5420178C1F3810125
:1087A000012949D002294AD046F660512181A4F816
:1087B000A820B0F9243089B24B439B13A4F8A4300D
:1087C000B0F90E0000237043B0FBF1F0216DC0F34F
:1087D000D100C1EBC101C90200EB91302065F01757
:1087E000810341EA9641B003F7F79CFCB4F8AA1064
:1087F000C1EBC101C902C00800EB9130A4F8AA0086
:10880000616C206F0844206794F87420521CD2B227
:1088100084F87420082A05D3C008A4F8760084F8E8
:10882000745025673748384EC3885A0633D498F8B1
:108830000F20022A06D02CE045F6C051B6E746F2DA
:108840009051B3E7B26840F69916B24221DD94F830
:10885000382094F88E60B2420CD084F88E2094F8C0
:108860003D2002F00106C2F34002964202D1A4F874
:108870008A5004E0B4F88A20B2F5966F05D2B4F8B5
:108880008A00401CA4F88A0005E043F08002C28000
:1088900001E0A4F88A50114894F83F30B8300C2B0E
:1088A00001D2C57400E0C774174A0F4C41F2482644
:1088B00092F83C20B4F8824041F2504C0C2B0AD381
:1088C000B14208DB012A06D0614502DD002C00D14F
:1088D0008774BDE8F0818574FBE700004801002043
:1088E0003407002000040040B00200204564BD01B0
:1088F00000209C40133B334002040020030400206E
:10890000D8040020640A00204005002070B5284CDF
:10891000284821880288511A89B23E2947D3008805
:1089200020802548808B254D800228606969284673
:1089300088472349A868FDF767F822496060CB881B
:108940005A072ED40022B0F1F05F0FD9E089B0F5BC
:10895000FA7F08D943F00400C8801B48017821F051
:10896000020101701CE0401CE0811AE0B0F1D25F0E
:108970000CD94FF4F031A1EB10308003C910B0FBDB
:10898000F1F0206100280CDA22610AE0B0F1C85F42
:1089900003D94FF48040206103E023F00400C88035
:1089A000E281D4E90401884200DB0846A06170BD81
:1089B0005C0C002034070020B00200209C06002040
:1089C00040970008640A0020EA05002005494FF49A
:1089D00080404861086188610348C18821F4827140
:1089E000C18070475C0C0020640A00202DE9F04132
:1089F000384C394E394F207841F23331C2074FF0AD
:108A000000050CD0A28962B394F90700002800DAAF
:108A10004042C0B2032829D240F2AE702AE0A570CD
:108A2000E5732F4AE571A58192F83830237220F062
:108A30000800A18040F0020020703D867560B5609E
:108A4000F560116D490005D041F68461A18140F0C7
:108A500010002070C0B240F0010020706574BDE8C5
:108A6000F081658120F01000207015E0042803D209
:108A700040F6510060810FE0052802D240F69910BF
:108A8000F8E740F6CC42062803D3072801D308288C
:108A900001D2628100E0618197F89D0098B9B088A9
:108AA000102301B2B4F90A003622FBF7F5FF70601B
:108AB000F168401AB1680844B060B6F90010484344
:108AC000C013F0603886388E10B10120A070C6E760
:108AD000A570C4E7780C0020B4060020B002002086
:108AE000480100202DE9F041554C2678F0077CD054
:108AF0005448217A544D90F8380081427BD0534A33
:108B00002346DFF84CC1575C93F90E2093F90730E8
:108B1000874203D01CF80170874213D146F0020649
:108B20005B1C26705BB2E3711CF80110814201D11D
:108B30005B1CE37194F90710062901DD0621E17140
:108B4000521C1CE0434F17F801C0434F844503D02B
:108B500017F801C0844513D126F002065B1E26706B
:108B60005BB2E371795C814201D15B1EE37194F9E0
:108B700007306FF005018B4200DAE171521EA273DB
:108B8000207294F907108A1C042A02D941F68462E3
:108B9000A2812C4A012912780ADD2B4B56079B68CB
:108BA00002D543F0080301E023F00803AB606070D6
:108BB000B1F1FF3F09DA5107A96802D521F0080198
:108BC00001E041F00801A9606070F9F79DFBA07811
:108BD000012810D121488068A3280CDA94F90700F5
:108BE000022803DD0220E07105E01EE06FF00101C4
:108BF000884200DAE171A089002630B1401E0004ED
:108C0000000CA08101D1E671A673E87B04280CD08A
:108C1000B5F93010512341220020FBF73DFF288693
:108C2000002802D1E07B10B1A670BDE8F0810C48AD
:108C300006700C480670207820F001002070F4E7E0
:108C4000780C002048010020B0020020389800086D
:108C50003E9800084A9800085098000840050020F7
:108C6000480700202B070020743F713D9B3BED39E6
:108C70006238F436A13565343F332A322731333038
:108C80004C2F722EA32DDF2C242C722B00000036CB
:108C90001C070038AA0A003AAA0A003CCC0C003E85
:108CA000CC0C0040380E0042380E0044380E00460E
:108CB000380E0048380E004AC711004CC711004E4C
:108CC000C7110050C7110052C7110054C7110056F8
:108CD000C7110058C711005AC711005CC711005EC8
:108CE000C7110060C7110062C7110064C711006698
:108CF000C7110068C711006A000000362202003860
:108D00008E03003AB005003CD207003EF409004053
:108D1000160C0042380E00445B100046C711004894
:108D20003313004A9F14004C9F14004E0B16005042
:108D300077170052771700547717005677170058A7
:108D40007717005A7717005C7717005E7717006077
:108D50007717006277170064771700667717006847
:108D60007717006A0000003600000038B600003AAD
:108D70006C01003C2202003ED80200408E030042FB
:108D800044040044FA040046B00500486606004A60
:108D90001C07004CD207004E880800503E090052C4
:108DA000F4090054AA0A0056600B0058160C005A29
:108DB000CC0C005C820D005E380E0060EE0E00628E
:108DC000A40F00645B10006611110068C711006AEF
:108DD0000000003400000036000000380000003AB7
:108DE0000000003C0000003E000000400000004287
:108DF0000000004400000046000000480000004A57
:108E00000000004C0000004E000000500000005226
:108E10000000005400000056000000580000005AF6
:108E20000000005C0000005E0000006000000062C6
:108E300000000064000000660000006844145858F8
:108E400058701111585858704111585848701114E1
:108E5000485858701411584858700020007200206B
:108E600000700020006E0020006C0020006A0020CE
:108E700000680020006600200064002000620020DE
:108E800000600020005E0020005C0020005A0020EE
:108E900000580020005600200054002000520020FE
:108EA00000500020004E0020004CA320004AA320C8
:108EB000004847210046EB210044EB2100428F226D
:108EC00000408F22003E7A24003C7A24003A662635
:108ED0000038512800343D2A0030702D002CA3307A
:108EE00000287A34002451380020CC3C001C00407B
:108EF000001800400014004000100040000C00402A
:108F000000080040000400400000000001020304CB
:108F1000050005000102030401040003050200002E
:108F2000F001000036010000F8000000BA00000067
:108F30007C0000007C0000007C0000004114141143
:108F400011144411141441110000290052007B0037
:108F5000A400CC00F5001E01470170019901C20177
:108F6000EA0113023C0265028E02B602DF02080328
:108F7000300359038203AA03D303FB0324044C04E4
:108F800075049D04C504EE0416053E0567058F05AE
:108F9000B705DF0507062F0657067F06A706CE068C
:108FA000F6061E0746076D079507BC07E4070B0882
:108FB000320859088108A808CF08F6081D09440995
:108FC0006A099109B809DE09050A2B0A520A780ACA
:108FD0009E0AC40AEA0A100B360B5C0B820BA80B24
:108FE000CD0BF30B180C3E0C630C880CAD0CD20CA3
:108FF000F70C1C0D410D650D8A0DAF0DD30DF70D4E
:109000001C0E400E640E880EAC0ECF0EF30E170F22
:109010003A0F5E0F810FA40FC70FEA0F0D1030102B
:10902000531075109810BA10DD10FF102111431164
:1090300065118711A911CA11EC110D122E125012CF
:1090400071129212B312D412F4121513361356136E
:1090500076139613B713D713F61316143614561443
:1090600075149414B414D314F214111530154E154C
:109070006D158C15AA15C815E7150516231641168A
:109080005F167C169A16B716D516F2160F172C1700
:10909000491766178317A017BC17D917F5171118AA
:1090A0002E184A18661881189D18B918D418F01887
:1090B0000B19261942195D1978199219AD19C81999
:1090C000E219FD19171A311A4C1A661A801A991AE0
:1090D000B31ACD1AE61A001B191B331B4C1B651B58
:1090E0007E1B971BAF1BC81BE11BF91B121C2A1C04
:1090F000421C5A1C721C8A1CA21CBA1CD21CE91CE1
:10910000011D181D301D471D5E1D751D8C1DA31DE5
:10911000BA1DD01DE71DFD1D141E2A1E401E571E20
:109120006D1E831E981EAE1EC41EDA1EEF1E051F86
:109130001A1F2F1F451F5A1F6F1F841F991FAE1F15
:10914000C21FD71FEC1F002000006400C9002D01C2
:109150009201F7015B02C00224038903ED0352046C
:10916000B6041A057F05E3054706AB060F0773072C
:10917000D7073B089F0802096609C9092D0A900A0A
:10918000F30A560BB90B1C0C7F0CE20C440DA60D18
:10919000090E6B0ECD0E2F0F900FF20F5310B4105F
:1091A00015117611D71138129812F8125813B813F6
:1091B00018147714D61435159415F3155116B016E6
:1091C0000E176B17C91726188318E0183D1999193F
:1091D000F519511AAD1A081B631BBE1B181C731C12
:1091E000CD1C261D801DD91D321E8A1EE31E3B1F6D
:1091F000921FEA1F41209820EE2044219A21EF215E
:1092000045229922EE2242239623E9233C248F24EF
:10921000E22434258525D72528267826C826182730
:109220006827B72706285428A228EF283D2989292E
:10923000D629222A6D2AB82A032B4D2B972BE12BF6
:109240002A2C722CBB2C022D4A2D912DD72D1D2E90
:10925000632EA82EEC2E302F742FB82FFA2F3D300E
:109260007F30C030013141318131C13100323F3274
:109270007D32BA32F73234337033AC33E7332234D1
:109280005C349534CE3407353F357735AE35E4352B
:109290001A3650368536B936ED362037533786378D
:1092A000B737E937193849387938A838D738053900
:1092B00032395F398B39B739E2390D3A373A603A8A
:1092C000893AB23ADA3A013B283B4E3B733B983B32
:1092D000BD3BE03B043C263C483C6A3C8B3CAB3C01
:1092E000CB3CEA3C093D273D443D613D7D3D993DF8
:1092F000B43DCE3DE83D013E1A3E323E493E603E21
:10930000763E8C3EA13EB53EC93EDC3EEF3E013F7F
:10931000123F233F333F433F513F603F6E3F7B3F10
:10932000873F933F9E3FA93FB33FBC3FC53FCD3FE3
:10933000D53FDC3FE23FE83FED3FF13FF53FF93FEE
:10934000FB3FFD3FFF3FFF3FFF3F0000E7382C356D
:10935000002020EF2037202333202620210000800A
:1093600002000400080010000002000400080400CD
:1093700000020004000800100020004000800400EB
:1093800000000080000000400000002000000010ED
:1093900000000008000000040000000200000001BE
:1093A00000008000000040000000200000001000CD
:1093B000000008000000040000000200000001009E
:1093C0000080000000080140000C0140000C01403A
:1093D000000C0140000C0140000C0140000C014059
:1093E000000C01400010014000100140001001403D
:1093F0000010014000100140001001400010014029
:10940000001001400014014004080140040C014018
:10941000040C0140040C0140040C0140040C014008
:10942000040C0140040C01400410014004100140F0
:1094300004100140041001400410014004100140D8
:1094400004100140041001400414014008080140C8
:10945000080C0140080C0140080C0140080C0140B8
:10946000080C0140080C0140080C014008100140A4
:109470000810014008100140081001400810014088
:109480000810014008100140081001400814014074
:109490000C0801400C0C01400C0C01400C0C01406C
:1094A0000C0C01400C0C01400C0C01400C0C014058
:1094B0000C1001400C1001400C1001400C10014038
:1094C0000C1001400C1001400C1001400C10014028
:1094D0000C14014010080140100C0140100C014018
:1094E000100C0140100C0140100C0140100C014008
:1094F000100C0140101001401010014010100140EC
:1095000010100140101001401010014010100140D7
:109510001010014010140140000000000000000085
:1095200000000000000000000000000014080140DE
:10953000140C0140140C0140140C0140140C0140A7
:10954000140C0140140C0140140C01401410014093
:109550001410014014100140141001401410014077
:109560001410014014100140141001401414014063
:1095700000000000000000000000000000000000EB
:1095800000000000FFFFFF0F0FFFFFFFFFF0FFFFD6
:10959000FF0FFFFFFFFFF0FF0FFFFFFFFFF0FFFFD9
:1095A000FF0FFFFFFFF0FFFF0FFFFFFFFFF0FFFFC9
:1095B000FF0FFFFFFFFFF0FFFFFF0FFFFFFFFFF0B9
:1095C000FFFFFF0FFFF0FFFF000000404000000022
:1095D0000004000000400000000004004000000003
:1095E00000040000004000000004000040000000F3
:1095F00000040000004000000000040000004000E3
:109600000000000400000040000400000000008092
:10961000800000000008000000800000000008003A
:10962000800000000008000000800000000800002A
:10963000800000000008000000800000000008001A
:10964000000080000000000800000080000800000A
:1096500000000020200000000002000000200000A8
:1096600000000200200000000002000000200000B6
:1096700000020000200000000002000000200000A6
:109680000000020000002000000000020000002096
:109690000002000000000060600000000006000002
:1096A00000600000000006006000000000060000EE
:1096B00000600000000600006000000000060000DE
:1096C00000600000000006000000600000000006CE
:1096D0000000006000060000008002000400080096
:1096E000100000020004000804000002000400084A
:1096F000001000200040008004000000FF7FFFFFFA
:10970000FDFFFFFFFBFFFFFFF7FFFFFFEFFFFFFF87
:10971000FFFDFFFFFFFBFFFFFFF7FFFFFBFFFFFF6B
:10972000FFFDFFFFFFFBFFFFFFF7FFFFFFEFFFFF67
:10973000FFDFFFFFFFBFFFFFFF7FFFFFFBFFFFFF1D
:109740000000401F7A1903000000001E8976030004
:109750000000C01C3BDF03000000801BD157040049
:109760000000401A9FE00400000000199E7B0500E5
:109770000000C017E42C0600000080160DF806005B
:109780000000401593DE07000000001408E6080002
:109790000000C012B1110A000000801101650B0029
:1097A00000004010E6E30C000000000F46940E009D
:1097B0000000C00D467710000000800CB08F120032
:1097C0000000400BD2DE14000000000A5E631700A8
:1097D0000000C008601A1A000000800726FC1C0068
:1097E0000000400600002000000000057A19230058
:1097F0000000C003D539260000008002585129001E
:1098000000004001764F2C000000000046252F008C
:109810000000C0FE2AC63100000080FDA1283400EF
:10982000000000FB4B1F3800000080F829053B00BA
:10983000000000F6EFFE3C000102030405000203F5
:1098400004050001030405000102050001020304F0
:1098500004050001020355050010AA1A5525003021
:10986000AA3A0000AA0A55150020AA2A5535FF3F3A
:10987000909800080000002060070000E40600083F
:109880008899000860070020D809000034670008A4
:1098900045020406082D01020304040548060708D2
:1098A00009134D2B1B086104211355152A40061975
:1098B0000801A713C73D1B08ED041AE7040125178B
:1098C000020604050103148020FF8BAA0A0201A4EA
:1098D00015AA0A551500085920AA2A5535FF3F0731
:1098E0002D03010504060203127C1573FFFF04FF1C
:1098F0008080010129025F6402130A13AD6A5208D5
:109900001201100C050406020301010307050528D6
:109910000B010203040206070303040C3D070604BF
:109920000509191F191904310506060B14AA1A0294
:10993000312E40FD3969260211042F405F020C26AA
:10994000405B262ACD55155515123902017F0316A5
:10995000D0071AFF01013B0261AA0C12080108A8F6
:10996000147F993F23403313B1720A1608DC912209
:109970000312100A17401C12600A16901B014D13A7
:08998000C16A020008000000AA
:020000040800F2
:10FC00004A46545A594D46312D4E3330202020203B
:10FC1000050406020301AA0AAA0AAA0AAA0AAA0A4B
:10FC2000AA0ADE3F00100000FF0131000201664613
:10FC300000400040513800400040004000400101B9
:10FC400000400040FF387B257B257B25FF003333B8
:10FC50000201401F00016626B81E6626FFFFFFFF57
:10FC6000FFFF01010100010000000300000200008D
:04FC70000000AA5591
:04000005080000ED02
:00000001FF
